:100000000C94D0020C94F8020C94F8020C94F802B0
:100010000C94F8020C94F8020C94F8020C94F80278
:100020000C94F8020C94F8020C94F8020C94F80268
:100030000C94F8020C94F8020C94F8020C94F80258
:100040000C94B52E0C94F8020C94B2300C94003140
:100050000C94F8020C94F8020C94F8020C94F80238
:100060000C94F8020C94F8021A1BF41ABF1C9B1B88
:10007000851B6C1C061BBF1C3E1BEB1AFD1A5B1C70
:10008000881B5D1BA81C0F1B311BD21AAF1C471C01
:10009000501C631C5E1CBF1C910395039A039E03B6
:1000A000A803AD03B403B903BF03C403C903CE035C
:1000B000D503DD03E503EB03F003F60302040A04B2
:1000C0000F0416041D042504485454502F312E30BB
:1000D0002034303120556E617574686F72697A65AD
:1000E000640A436F6E74656E742D547970653A209E
:1000F000746578742F68746D6C0A3C68313E3430D6
:100100003120556E617574686F72697A65643C2F31
:1001100068313E0057616B652075700A004D61695A
:100120006E74656E616E63650A00206D730A004D22
:100130006F64652045434F200046696E2064656CFE
:100140006573746167650A004D6F64652064656C52
:100150006573746167650A00537263206164647239
:10016000657373203A20004C6E646B205472616397
:1001700065722076302E38652C202863294C652046
:100180004E6574206475204B65726D657572203202
:100190003031332D323031360A002C2047617465FE
:1001A0007761793A20002C204E65746D61736B3A4B
:1001B0002000495020616464726573733A20002006
:1001C0006D560A00206D562C2056696E3A2000208C
:1001D00062797465732C205663633A200046726519
:1001E00065206D656D6F72793A20006261636B20E6
:1001F000746F203139322E3136382E312E32350A95
:1002000000646F6E650A0052657175657374696E7E
:10021000672049502041646472657373202E2E2E2E
:1002200020004661696C656420746F2061636365BA
:10023000737320454E4332384A36300A00454E43E8
:1002400032384A36302076657273696F6E200064EA
:100250006F6E650A00496E697420454E4332384A14
:100260003630202E2E2E004D6F6465206465627539
:10027000670A00436F6D6D616E64203A20003C6830
:10028000313E323030204F4B3C2F68313E00556EAE
:10029000617574686F72697A656420616363657300
:1002A000730A005365742054696D6520004D6F64B6
:1002B000652045434F206465736163746976650A00
:1002C000004D616E71756520706172616D6574724B
:1002D00065730A0020636172616374657265730AF5
:1002E000005265637520000A3C2F626F64793E0AF4
:1002F0003C2F68746D6C3E0A003C68746D6C3E3C2B
:10030000686561643E3C7469746C653E4C6E646BF8
:10031000205472616365723C2F7469746C653E3C55
:100320002F686561643E0A003C626F64793E3C68F8
:10033000313E4C6E646B2054726163657220766549
:100340007273696F6E2076302E38653C2F68313EAF
:100350000A00485454502F312E3020323030204F74
:100360004B0D0A436F6E74656E742D547970653A47
:1003700020746578742F68746D6C0D0A5072616713
:100380006D613A206E6F2D63616368650D0A0D0A19
:1003900000414343004144445200434D440044451E
:1003A0004C4553544147450044554D500045455038
:1003B000524F4D004741544500484953544F004C5B
:1003C0004F4144004D414341004D41534B004D4589
:1003D0004D4F5259004D455355524553004D4F44D2
:1003E0004545434F00504152414D00504F5254003B
:1003F00052455345540053455249414C444542559A
:1004000047005354414E4442590054494D4500550C
:100410005054494D450056494E4D415800564F4C99
:1004200054414745005741544348444F4700000159
:100430000800060400014500008200004000200D75
:100440000A436F6E74656E742D547970653A20613D
:1004500070706C69636174696F6E2F782D77777730
:100460002D666F726D2D75726C656E636F64656459
:100470000D0A0D0A00436F6E74656E742D4C656E27
:100480006774683A20000D0A557365722D416765DF
:100490006E743A204574686572536869656C642FA0
:1004A000312E360D0A4163636570743A202A2F2A73
:1004B0000D0A436F6E6E656374696F6E3A20636CEC
:1004C0006F73650D0A000D0A0020485454502F31F7
:1004D0002E310D0A486F73743A2000504F53542048
:1004E0000020000D0A557365722D4167656E743AE0
:1004F000204574686572536869656C642F312E36C7
:100500000D0A4163636570743A20746578742F68CE
:10051000746D6C0D0A436F6E6E656374696F6E3A2D
:1005200020636C6F73650D0A0D0A00204854545007
:100530002F312E310D0A486F73743A20004745540D
:10054000200000000000240027002A000000000016
:10055000250028002B0000000000230026002900B1
:100560000404040404040404020202020202030359
:100570000303030301020408102040800102040861
:1005800010200102040810200000000700020100F2
:1005900000030406000000000000000000076E32A7
:1005A00011241FBECFEFD8E0DEBFCDBF15E0A0E025
:1005B000B1E0ECEFFAE602C005900D92A83AB1075F
:1005C000D9F717E0A8EAB5E001C01D92A03FB10736
:1005D000E1F715E0C0EAD5E004C02297FE010E94D1
:1005E0004135CC39D107C9F70E94C4320C947C350F
:1005F0000C940000A0E0B0E0E0E0F3E00C944D3596
:10060000EC01A880B980CA80DB80A114B104C104C8
:10061000D10441F484E2A82E89EDB82E8BE5C82ED2
:1006200087E0D82EC601B5012DE133EF41E050E05F
:100630000E94243527EA31E440E050E00E94BC34B7
:100640007B018C01C601B5012DE133EF41E050E0A3
:100650000E942435CA01B9012CEE34EF4FEF5FEF51
:100660000E94BC346E0D7F1D801F911F97FF04C038
:100670006150704080409048688379838A839B836F
:100680009B013F77C901CDB7DEB7EAE00C9469352D
:100690000E94FA0208958BE291E00E94FA02089506
:1006A000A0E0B0E080932B0190932C01A0932D014A
:1006B000B0932E010895FC0105900020E9F7809584
:1006C00090958E0F9F1F0895FB01DC014150504013
:1006D00030F08D910590801919F40020B9F7881B2E
:1006E000990B0895DC0101C06D9341505040E0F733
:1006F0000895FB01DC014150504030F08D91019094
:10070000801919F40020B9F7881B990B0895EF920E
:10071000FF920F931F93CF93DF93EC01A0E0B0E023
:10072000EE24FF24870109C0F901EA0FFB1F808135
:10073000E80EF11C011D111D1196A617B707A4F3B1
:10074000452B69F09B01442737FD4095542FB70195
:10075000C8010E940235C901DA017C018D01D8016E
:10076000C701807F9070A070B07024E0B695A79507
:10077000979587952A95D1F78A3010F0895C01C04A
:10078000805DFE01E058FB4F80839E012F5F3F4F4D
:100790006E2D6F706A3010F0695C01C0605DF90108
:1007A000E058FB4F60832F5F3F4FF901E058FB4F4C
:1007B00080E280832F5F3F4FC901DF91CF911F916E
:1007C0000F91FF90EF900895EF92FF920F931F9378
:1007D000CF93DF93EC01FA0120E030E0EE24FF2418
:1007E00087010AC081919191A0E0B0E0E80EF91E66
:1007F0000A1F1B1F2F5F3F4F261737079CF39B01D4
:10080000442737FD4095542FC801B7010E94023597
:1008100079018A01D801C7016CE0B695A795979533
:1008200087956A95D1F78F708A3010F0895C01C086
:10083000805DFE01E058FB4F80839E012F5F3F4F9C
:10084000BB27A12F902F8F2D8F708A3010F0895CDD
:1008500001C0805DF901E058FB4F80832F5F3F4F5F
:10086000D801C701807F9070A070B07044E0B69549
:10087000A795979587954A95D1F78A3010F0895CAE
:1008800001C0805DF901E058FB4F80832F5F3F4F2F
:100890004E2D4F704A3010F0495C01C0405DF901A7
:1008A000E058FB4F40832F5F3F4FF901E058FB4F6B
:1008B00080E280832F5F3F4FC901DF91CF911F916D
:1008C0000F91FF90EF9008959C01DB01CA01FCE1BC
:1008D000B695A79597958795FA95D1F78A309105A2
:1008E00014F0895C01C0805DF901E058FB4F808302
:1008F0002F5F3F4FDB01CA0180709070A070BF7006
:100900008B2F9927AA27BB278A30910514F0895C81
:1009100001C0805DF901E058FB4F80832F5F3F4F9E
:10092000DB01CA0180709070A07FB070F4E1B695D1
:10093000A79597958795FA95D1F78A30910514F088
:10094000895C01C0805DF901E058FB4F80832F5F17
:100950003F4FDB01CA0180709070AF70B070CD0165
:10096000AA27BB278A30910514F0895C01C0805DFD
:10097000F901E058FB4F80832F5F3F4FDB01CA0135
:100980008070907FA070B070FCE0B695A7959795A9
:100990008795FA95D1F78A30910514F0895C01C0EA
:1009A000805DF901E058FB4F80832F5F3F4FDB01F3
:1009B000CA0180709F70A070B070892F9A2FAB2FE2
:1009C000BB278A30910514F0895C01C0805DF90174
:1009D000E058FB4F80832F5F3F4FDB01CA01807FD0
:1009E0009070A070B07074E0B695A79597958795B4
:1009F0007A95D1F78A30910514F0895C01C0805D49
:100A0000F901E058FB4F80832F5F3F4F4F705070CC
:100A10004A30510514F0495C01C0405DF901E058CD
:100A2000FB4F40832F5F3F4FF901E058FB4F80E2BF
:100A300080832F5F3F4FC9010895DC01FC01E05A1C
:100A4000FE4FE0818E2F80538A3038F081518630FE
:100A500010F080E002C08E2F8753982F9295907FE0
:100A6000A05ABE4F1196EC918E2F80538A3010F40D
:100A7000892B08958E2F8154863010F080E00895E0
:100A80008E2F8753892B0895FC0150814181A82F17
:100A9000FC0170E062507040B0E131E416C0228188
:100AA00090E0852F880F47FD8F5F440F27FD4F5F34
:100AB00057FD02C0582F03C0582F5B2743279F5F65
:100AC000983011F0220FEDCF31968E2F8A1B90E0D7
:100AD0008617970724F3952F80E0242F30E0282BEA
:100AE000392BC90108952F923F924F925F926F92D6
:100AF0007F928F929F92AF92BF92CF92DF92EF92AE
:100B0000FF920F931F93DF93CF93CDB7DEB7289754
:100B10000FB6F894DEBF0FBECDBF809120048B3E90
:100B200009F055C180912104803909F050C18091AC
:100B300022048B3E09F04BC180912304803909F0D7
:100B400046C1809124048B3E09F041C18091250467
:100B5000803909F03CC183E696E09C838B83EFE407
:100B6000F6E0FA83E9836BE3262E66E0362E57E241
:100B7000652E56E0752E43E1842E46E0942E3FE923
:100B8000A32E36E0B32E25E9C22E26E0D22E9BE816
:100B9000E92E96E0F92E01E816E067E776E047ECEB
:100BA00056E02DEB36E083EB96E098878F83A9EA39
:100BB000B6E0EFEFF5E0FE83ED8388E0482E512CA0
:100BC000EB81FC8180899189938B828BE981FA8109
:100BD00080899189938B828BF10180899189938B94
:100BE000828BF30180899189938B828BF4018089B8
:100BF0009189938B828BF50180858187F6018085B1
:100C00008187F70180858187F80180858187FB01D5
:100C100080858187FA0180858187F90180858187B8
:100C2000EF81F8858085818718968C9118971996A1
:100C30008C931997ED81FE8180899189938B828BAA
:100C40000894410851088B819C8102979C838B8377
:100C5000E981FA813297FA83E9838EEF9FEF280EBC
:100C6000391E680E791E880E991E0894A108B108D5
:100C70000894C108D1080894E108F1080150104017
:100C8000615070404150504021503040EF81F88514
:100C90003197F887EF8311978D819E8102979E830C
:100CA0008D839FEF49169FEF590609F089CF9091E8
:100CB0002A0480E02091290430E0822B932B90932A
:100CC00064068093630690912C0480E020912B04AD
:100CD00030E0822B932B9093500680934F06909197
:100CE000300480E020912F0430E0822B932B9093EE
:100CF0003C0680933B069091320480E020913104C1
:100D000030E0822B932B90932806809327069091B6
:100D1000340480E02091330430E0822B932B9093B5
:100D20001406809313068091350480939F0680916A
:100D30003604809395068091370480938B068091CA
:100D400038048093810680913904809377068091DE
:100D50003A048093C70680913B048093BD0680913E
:100D60003C048093B30680913D048093A906909142
:100D70003F0480E020913E0430E0822B932B90933F
:100D800000068093FF0510914104009142041092E7
:100D900042041092410486E294E06DE10E94440511
:100DA00010934104009342049093440480934504BB
:100DB0008091EC059091ED0501969093ED0580935F
:100DC000EC051092B3051092B2051092800428969B
:100DD0000FB6F894DEBF0FBECDBFCF91DF911F914C
:100DE0000F91FF90EF90DF90CF90BF90AF909F90CA
:100DF0008F907F906F905F904F903F902F900895CD
:100E000080EF95E00E94F52C08950F931F93CF93E8
:100E1000DF938C01C0E0D0E0F801EC0FFD1F8AEBFE
:100E200097E060814AE050E00E94B433C330D105BE
:100E300031F08AEB97E060E071E00E945634219631
:100E4000C430D10549F7DF91CF911F910F910895DB
:100E5000AC0180EF95E060E671E027EE32E00E94A1
:100E6000A52D0895EF92FF920F931F93AC0100EF11
:100E700015E070E6E72E71E0F72EC801B70129EF03
:100E800032E00E94A52DAC01C801B70128E233E091
:100E90000E94A52D1F910F91FF90EF90089580EF74
:100EA00095E060E671E040E050E022E533E00E942A
:100EB000A52D08958EE480937C0062E070E080E0D0
:100EC00090E00E940B2F80917A00806480937A00DA
:100ED00080917A0086FDFCCF8091780090E0A0E0C0
:100EE000B0E060917900362F20E0442737FD40952F
:100EF000542F282B392B4A2B5B2B60E070E381E1C8
:100F000090E00E942435CA01B9010895CF93DF9380
:100F1000EC010CC06A3029F48AEB97E00E9405339B
:100F200004C08AEB97E00E942C322196FE01649166
:100F3000662381F7DF91CF9108950F931F93CF938D
:100F4000DF938C01E091AC05EE2309F400C1209100
:100F5000A805222369F48091A905882349F480918A
:100F6000AA05882329F48091AB05882309F4EFC0F2
:100F700040E0A0E08A2F90E0880F991F50E04E17C4
:100F800008F451E0A52FA82B4F5F483099F760E097
:100F9000862F90E0880F991F50E04E1708F451E01B
:100FA000652F682B4F5F403199F770E0872F90E0F5
:100FB000880F991F50E04E1708F451E0752F782BD9
:100FC0004F5F483199F780E090E0880F991F50E01B
:100FD0004E1708F451E0582B852F4F5F4032A1F790
:100FE000F801E05AFE4F8081C82FD0E08A2F90E0B0
:100FF0008C239D2330E08217930729F5862F90E0FC
:10100000218130E0822393232091A90530E08217CB
:101010009307C9F4872F90E0228130E08223932345
:101020002091AA0530E08217930769F4852F90E09C
:10103000238130E0822393232091AB0530E0821797
:10104000930709F484C0E091B105EE2309F47CC054
:101050002091AD05222369F48091AE05882349F4DF
:101060008091AF05882329F48091B005882309F485
:101070006BC0F72F40E08F2F90E0880F991F50E052
:101080004E1708F451E0F52FF82B4F5F483099F7D1
:10109000672F862F90E0880F991F50E04E1708F4B5
:1010A00051E0652F682B4F5F403199F7872F90E013
:1010B000880F991F50E04E1708F451E0752F782BD8
:1010C0004F5F483199F750E0852F90E0880F991FC6
:1010D00050E04E1708F451E0A52FA82B5A2F4F5F70
:1010E000403291F78F2F90E08C239D2330E08217C0
:1010F000930751F5862F90E0F801E05AFE4F2181C9
:1011000030E0822393232091AE0530E082179307CD
:10111000D9F4872F90E0228130E08223932320911D
:10112000AF0530E08217930779F4C0E0D0E08A2F52
:1011300090E0238130E0822393232091B00530E0BA
:101140008217930731F403C0C0E0D0E002C0C1E0D1
:10115000D0E08091B6059091B705892B31F02097AA
:1011600021F48EE892E00E948607CE01DF91CF91B4
:101170001F910F91089580915E0190915F010397F7
:1011800081F482E090E090935F0180935E01809112
:10119000B6059091B705892B21F08DEA92E00E9467
:1011A00086070895AF92BF92CF92DF92EF92FF929F
:1011B0000F931F93CF93DF935C014091D106509121
:1011C000D2064115510579F0C091D306D091D406CD
:1011D000FE01EE0FFF1FE856FF4F659174910E94CC
:1011E0006403892B19F1CC24DD24E7E1EE2EF12CE8
:1011F000E601CE0DDF1DD595C795D093D406C093DB
:10120000D306FE01EE0FFF1FE856FF4F0591149124
:10121000C8010E945B03AC019093D2068093D10673
:10122000C501B8010E946403009719F4FE01B0964D
:1012300011C0181619062CF46E010894C11CD11C9B
:1012400004C07E010894E108F108EC14FD0484F662
:10125000E0E0F0E0CF01DF91CF911F910F91FF907F
:10126000EF90DF90CF90BF90AF900895CF92DF9234
:10127000EF92FF920F931F93CF93DF93C0905E0185
:10128000D0905F010E94072E029709F0E2C00E94F1
:10129000FD2E2091CA053091CB054091CC0550918F
:1012A000CD05621B730B840B950B615A7B4B8D40F4
:1012B000904008F4CEC080915E0190915F011816B5
:1012C00019060CF0C6C08091EC059091ED050997C8
:1012D0000CF4BFC00E94FD2E6093CA057093CB052D
:1012E0008093CC059093CD05C091EC05D091ED0590
:1012F000CB30D10514F0CAE0D0E0E3E6F6E060E0E0
:1013000070E020E030E040E050E00AC0819191912F
:10131000A0E0B0E0280F391F4A1F5B1F6F5F7F4FAF
:101320006C177D079CF3CA01B9012AE030E040E068
:1013300050E00E94BC349E01442737FD4095542F55
:101340000E94023579018A0120E030E040E050E05F
:1013500008C0F901ED54F94F8081480F511D2F5FEE
:101360003F4F2C173D07ACF320E030E060E070E029
:1013700008C0F901EF57F94F8081680F711D2F5F89
:101380003F4F2C173D07ACF380914C0190914D01DC
:10139000A0E0B0E0E816F9060A071B07A8F04C1712
:1013A0005D0791F480915001909151019C01429F01
:1013B000C001439F900D529F900D1124681779072B
:1013C00018F081E0C82ED12C80914E0190914F01F0
:1013D000A0E0B0E0E816F9060A071B0788F0452BE5
:1013E00079F080915201909153019C01C29FC001FC
:1013F000C39F900DD29F900D11246817790748F56F
:1014000080915E0190915F01019719F51092E605B8
:101410001092E7051092E8051092E9051092E20596
:101420001092E3051092E4051092E5051092DE0596
:101430001092DF051092E0051092E1051092DA0596
:101440001092DB051092DC051092DD0502E0C02E43
:10145000D12C80915E0190915F01039709F062C0E9
:101460008091D6059091D705A091D805B091D90566
:10147000805C944DA140B04008F454C00E94FD2E01
:101480002091CE053091CF054091D0055091D105E6
:10149000621B730B840B950B2091D6053091D705F9
:1014A0004091D8055091D905220F331F441F551F75
:1014B0002617370748075907A8F51092E605109236
:1014C000E7051092E8051092E9051092E2051092E6
:1014D000E3051092E4051092E5051092DE051092E6
:1014E000DF051092E0051092E1051092DA051092E6
:1014F000DB051092DC051092DD0580EF95E00E947F
:10150000F92C0E94FD2E6093D2057093D305809331
:10151000D4059093D5051092EB051092EA05B2E040
:10152000CB2ED12CC601DF91CF911F910F91FF904F
:10153000EF90DF90CF9008950E94072E805D8093FA
:1015400080048091EC059091ED05409734F08FE098
:1015500090E09093ED058093EC058091EC059091DF
:10156000ED058A30910514F0895C01C0805D80939F
:10157000810480915E01805D809382048091EA0500
:10158000805D8093830480E2809384040E94422ED5
:10159000AB01BC0185E090E00E94640408950E94C4
:1015A0004F070E943207AC0180EF95E060E671E0E2
:1015B00020E834E00E949F2D0E9428070895EF92B2
:1015C000FF920F931F93CF93DF937C010E94422ED3
:1015D0000E94072E805D809380048091EC0590919D
:1015E000ED05409734F08FE090E09093ED05809307
:1015F000EC058091EC059091ED058A30910514F091
:10160000895C01C0805D8093810480915E01805D72
:10161000809382048091EA05805D8093830480E258
:10162000809384040E94422EAB01BC0185E090E0CF
:101630000E946404FC011E141F0434F5C0E2D4E0CF
:10164000DC01A058BB4F20E29881892F82958F70D2
:101650008A3010F0895C01C0805D8C93892F8F7077
:101660008A3010F0895C01C0805D11968C931197CF
:1016700012962C9312972196139684E0C834D807BB
:1016800019F7E858FF4F6DC06091EC057091ED05BA
:10169000161617060CF065C0EB016B30710514F0DF
:1016A000CAE0D0E0CF01BE0143E656E00E94E40369
:1016B000BE014FE456E00E94E403BE014BE356E056
:1016C0000E94E403BE0147E256E00E94E403BE012B
:1016D00043E156E00E94E403BE014FEF55E00E9453
:1016E000E403BE0140E050E02FE936E00E948703AA
:1016F000BE0140E050E025E936E00E948703BE01CC
:1017000040E050E02BE836E00E948703BE0141E054
:1017100050E021E836E00E948703BE0140E050E03F
:1017200027E736E00E948703BE0140E050E027EC47
:1017300036E00E948703BE0140E050E02DEB36E02A
:101740000E948703BE0140E050E023EB36E00E9498
:101750008703BE0141E050E029EA36E00E9487039A
:10176000FC01F093B505E093B405E058FB4F1082FF
:1017700080E691E00E94CF0A182F092F8091B605CC
:101780009091B7051816190694F481EE92E00E9424
:1017900086076091B2057091B3058AEB97E04AE045
:1017A00050E00E94243484ED92E00E948607EF28E6
:1017B00021F41092ED051092EC05812F902FDF910E
:1017C000CF911F910F91FF90EF9008955F926F92CC
:1017D0007F928F929F92AF92BF92CF92DF92EF92C1
:1017E000FF920F931F93CF93DF933C010E949C0ABB
:1017F000EC0185E10E94A92FAA24BB24812C24E0BE
:10180000922E00E010E0CC24DD24760190E2592EE7
:1018100064E170E080E090E00E940B2F85E10E947F
:10182000A92F9C01881599050CF44C010217130788
:101830000CF489016114710429F084E0A816B10444
:1018400009F047C0E3E0293E3E0764F0FE01E0589E
:10185000FB4FC90168EE73E00E94EF34605D608366
:10186000219603C02536310584F0FE01E058FB4F78
:10187000C90168EE73E00E94EF3464E670E00E94F4
:10188000EF34605D6083219603C02B3031057CF01E
:10189000FE01E058FB4FC90164E670E00E94EF349E
:1018A0006AE070E00E94EF34605D60832196FE0183
:1018B000E058FB4FC9016AE070E00E94EF34805DA0
:1018C0008083CE010196FC01E058FB4F5082EC0171
:1018D0002196C901AA2797FDA095BA2FC80ED91E37
:1018E000EA1EFB1E0894A11CB11CF7E0AF16B10460
:1018F00009F08ECF080D191DC801AA2797FDA095E4
:10190000BA2FC81AD90AEA0AFB0AA0904A01B09075
:101910004B01950140E050E0C701B6010E94BC3484
:1019200020E034E140E050E00E94023569017A0194
:10193000FE01E058FB4F88E28083219681E1C816C2
:1019400087E2D80680E0E80680E0F80680F08E01A5
:1019500000581B4FC701B60120E137E240E050E0DC
:101960000E940235205DF8012083219609C0F9EE1E
:10197000CF16F3E0DF06F0E0EF06F0E0FF06B0F090
:101980008E0100581B4FC701B60120E137E240E04D
:1019900050E00E94023528EE33E040E050E00E9423
:1019A0000235205DF8012083219606C0F5E6CF16AA
:1019B000D104E104F104B0F08E0100581B4FC701BF
:1019C000B60128EE33E040E050E00E94023524E604
:1019D00030E040E050E00E940235205DF8012083B5
:1019E000219606C0FBE0CF16D104E104F104A8F073
:1019F0008E0100581B4FC701B60124E630E040E0DD
:101A000050E00E9402352AE030E040E050E00E94C1
:101A10000235205DF801208321968E0100581B4F6E
:101A2000C701B6012AE030E040E050E00E940235F4
:101A3000605DF8016083CE010196FC01E058FB4F28
:101A400030E230830196FC01E058FB4F2DE6208305
:101A50000196FC01E058FB4F26E520830196FC012E
:101A6000E058FB4F29E22083DC011196672809F436
:101A70007DC0FD01E058FB4F3083CD010196FC0194
:101A8000E058FB4F2DE420830196FC01E058FB4F0A
:101A900021E620830196FC01E058FB4F28E72083D4
:101AA0000196FC01E058FB4F2AE320839C012F5F45
:101AB0003F4FF1E1AF16F7E2BF0668F0F901E058D9
:101AC000FB4FC50160E177E20E94DB34605D60831B
:101AD0002F5F3F4F05C089EEA81683E0B80688F057
:101AE000F901E058FB4FC50160E177E20E94DB3469
:101AF00068EE73E00E94DB34605D60832F5F3F4FD0
:101B000004C0E5E6AE16B10488F0F901E058FB4FD9
:101B1000C50168EE73E00E94DB3464E670E00E9469
:101B2000DB34605D60832F5F3F4F04C0FBE0AF1686
:101B3000B10480F0F901E058FB4FC50164E670E0A4
:101B40000E94DB346AE070E00E94DB34605D6083F9
:101B50002F5F3F4FF901E058FB4FC5016AE070E08D
:101B60000E94DB34805D8083D9011196A058BB4F61
:101B70001C9280E691E00E94CF0ADF91CF911F91E5
:101B80000F91FF90EF90DF90CF90BF90AF909F901C
:101B90008F907F906F905F9008950F931F93DF93C6
:101BA000CF9300D0CDB7DEB70E949C0AFC01E0586D
:101BB000FB4F26E420830196FC01E058FB4F22E70F
:101BC00020830196FC01E058FB4F25E62083019617
:101BD000FC01E058FB4F20830196FC01E058FB4FCD
:101BE0002AE320830196FC01E058FB4F20E220838A
:101BF0008C010F5F1F4F8091EC079091ED070097CC
:101C000011F480EF97E09E012F5F3F4F281B390BA7
:101C100087E22031380718F020E030E038C083E058
:101C2000293E38076CF0F801E058FB4FC90168EE17
:101C300073E00E94EF34605D60830F5F1F4F03C04D
:101C4000253631058CF0F801E058FB4FC90168EEEC
:101C500073E00E94EF3464E670E00E94EF34605D50
:101C600060830F5F1F4F03C02B30310584F0F801F4
:101C7000E058FB4FC90164E670E00E94EF346AE06F
:101C800070E00E94EF34605D60830F5F1F4FF801CA
:101C9000E058FB4FC9016AE070E00E94EF34805DBC
:101CA0008083F8013196DF01A058BB4F80E28C930E
:101CB0003196DF01A058BB4F82E68C933196DF014D
:101CC000A058BB4F89E78C933196DF01A058BB4FDA
:101CD00084E78C933196DF01A058BB4F85E68C9347
:101CE000EF57FB4F83E78083118280E691E00E94EB
:101CF000CF0A0F900F90CF91DF911F910F91089510
:101D00000F931F938C010E949C0AA80160E070E071
:101D10000E946404FC01E058FB4FAC014F5F5F4F31
:101D20000431110548F08FE48083FA01E058FB4F3D
:101D30008BE48083FA010EC085E48083FA01E058C9
:101D4000FB4F22E52083CA010196FC01E058FB4FBE
:101D50002083FC013196E058FB4F108280E691E031
:101D60000E94CF0A1F910F9108950F931F930E9415
:101D70009C0A8C010E94422EAB01BC018091BA05E5
:101D80009091BB05A091BC05B091BD05481B590BB6
:101D90006A0B7B0BC8010E946404FC019093B5059B
:101DA0008093B405E058FB4F108280E691E00E94DA
:101DB000CF0A1F910F9108957F928F929F92AF92B9
:101DC000BF92CF92DF92EF92FF920F931F93CF9328
:101DD000DF93EC01672B09F4D1C082E091E0BE01F2
:101DE00044E050E00E947903009709F0C7C0FC80EE
:101DF00005E010E0AA24BB2465011DC0C601B501A1
:101E00002AE030E040E050E00E94BC342F2D332720
:101E100027FD3095205330405901CC24B7FCC094A5
:101E2000DC2CA60EB71EC81ED91EFE01E00FF11F46
:101E3000F0800F5F1F4F8F2D80538A3018F40F30C2
:101E40001105E1F6B801615070406C0F7D1F87E00D
:101E500091E044E050E00E947903009721F0EE24E5
:101E6000FF24870147C0FE01E00FF11F738044E0AB
:101E7000842E912C800E911EEF01EE24FF24870109
:101E80001BC0C801B7012AE030E040E050E00E94EA
:101E9000BC34272D332727FD30952053304079015E
:101EA0000027F7FC0095102FE60EF71E081F191FDC
:101EB0007B800894811C911C872D80538A3028F4E4
:101EC000219629E182169104E4F2D801C7018857CE
:101ED0009040A040B040895A9B41A040B04030F0B3
:101EE00030EBE32E34E0F32E012D112DC801B701A4
:101EF0000E940C2E0E94072E892BB1F40E94FD2E09
:101F000028EE33E040E050E00E940235D601C501E2
:101F1000821B930BA40BB50B8093BA059093BB0562
:101F2000A093BC05B093BD05C601B5010E94152E56
:101F30008091B6059091B705892B01F183EA92E073
:101F40000E9486078AEB97E0B601A5012AE030E0FF
:101F50000E94A5338AEB97E06CE071E00E94563452
:101F60008AEB97E0B801A7012AE030E00E94A53390
:101F70008AEB97E06EE071E00E9459340E94B50E42
:101F8000DF91CF911F910F91FF90EF90DF90CF9055
:101F9000BF90AF909F908F907F900895CF92DF92E7
:101FA000EF92FF920F931F93CF93DF9391E0909363
:101FB00080048093810460938204A5EDB6E0C3E8B9
:101FC000D4E0E62FF0E09F012A0F3B1F02C08D9165
:101FD0008993A217B307D9F773E8E72E74E0F72EB9
:101FE000EE0EFF1ED7011C928F010C571B4FD8011C
:101FF0001C9255E0C52ED12CCE0EDF1EF601E05806
:10200000FB4F8FE780836B5F80E894E00E9444057C
:10201000F7019083D8018C93C0E0D0E08091EE0569
:102020009091EF05892B89F08091B6059091B705C5
:10203000892B59F48AEB97E06BEE0E942C328AEBE5
:1020400097E060E90E942C321AC08AEB97E06BEEB1
:1020500070E040E150E00E9424348AEB97E060E2B7
:102060000E94FD328AEB97E060E970E040E150E0C9
:102070000E9424348AEB97E060E20E94FD322196B0
:10208000C330D10559F6C0E8D4E000E010E08091FB
:10209000EE059091EF05892B51F08091B605909156
:1020A000B705892B21F48AEB97E0688112C08881FB
:1020B000803128F48AEB97E060E30E94FD328AEBDE
:1020C00097E0688140E150E00E94B4338AEB97E0EA
:1020D00060E20E942C320F5F1F4F2196C016D1067E
:1020E000B4F68091EE059091EF05892B39F080913F
:1020F000B6059091B7051816190624F48AEB97E0F7
:102100000E940533DF91CF911F910F91FF90EF90C7
:10211000DF90CF9008951092D506892B19F081E0B9
:102120008093D5061092D6068AEA61E00E94CE0F0F
:102130000895CF93DF93C0E0D0E088E197E0BE013F
:102140000E94F42DFE01E05EFB4F80832196C03497
:10215000D10599F710926004809120048D34A9F57F
:1021600080912104813489F5509122044091230407
:102170003091240420912504909126048091270415
:10218000552359F44423A9F4332399F4222389F4E1
:10219000992379F4882369F418C05F3F51F44F3FC5
:1021A00041F43F3F31F42F3F21F49F3F11F48F3F23
:1021B00061F050932F01409330013093310120930F
:1021C000320190933301809334018091280481344B
:1021D00021F580912904843401F580912A04843406
:1021E000E1F480912B048235C1F430912C042091CC
:1021F0002D0490912E0480912F043F3F31F42F3F06
:1022000021F49F3F11F48F3F41F03093350120932B
:1022100036019093370180933801809138048734D8
:1022200069F580913904813449F580913A04843507
:1022300029F580913B04853409F530913C042091C7
:102240003D0490913E0480913F04332339F42223CE
:1022500069F4992359F4882349F410C03F3F31F4BD
:102260002F3F21F49F3F11F48F3F41F0309339010C
:1022700020933A0190933B0180933C01809140046C
:102280008035B1F4809141048F3491F480914204FF
:10229000823571F480914304843551F48091440473
:1022A00090914504882311F4992311F090934901EA
:1022B00080914604813409F073C0809147048334CF
:1022C00009F06EC080914804833409F069C08091A0
:1022D0004904813309F064C040914A0430914B04B1
:1022E00020914C0490914D0450914E04852F8150C3
:1022F000803208F055C0442339F4332371F422238B
:1023000061F4992351F44CC04F3F39F43F3F29F415
:102310002F3F19F49F3F09F443C04093A805309321
:10232000A9052093AA059093AB055093AC05809125
:102330004F048134A9F580915004833489F580914C
:102340005104833469F580915204823349F54091F8
:1023500053043091540420915504909156045091A7
:102360005704852F81508032D8F4442339F4332325
:1023700069F4222359F4992349F412C04F3F31F4F0
:102380003F3F21F42F3F11F49F3F51F04093AD05A3
:102390003093AE052093AF059093B0055093B105EF
:1023A000809158048234E1F4809159048635C1F457
:1023B00080915A048934A1F480915B048E3481F4B5
:1023C00020915C0430915D04222311F4332341F009
:1023D000922F80E0830F911D90934B0180934A01CF
:1023E000809164048335E1F4809165048435C1F4FF
:1023F000809166048234A1F4809167048C3481F466
:102400002091680430916904222311F4332341F0B0
:10241000922F80E0830F911D90934F0180934E0186
:1024200080916A048335E1F480916B048F34C1F4A8
:1024300080916C048334A1F480916D04883481F41C
:1024400020916E0430916F04222311F4332341F064
:10245000922F80E0830F911D909351018093500142
:10246000809170048335E1F4809171048F34C1F45C
:10247000809172048334A1F4809173048C3481F4CC
:102480002091740430917504222311F4332341F018
:10249000922F80E0830F911D9093530180935201FE
:1024A000DF91CF9108954F925F926F927F928F92BA
:1024B0009F92AF92BF92CF92DF92EF92FF920F93D3
:1024C0001F93DF93CF9300D0CDB7DEB782E060E0FB
:1024D0000E94CB2F89E061E00E94CB2F82E00E9416
:1024E0005E30019711F40E94991085E10E94A92F96
:1024F00010E0662477246AE070E080E090E00E94BB
:102500000B2F85E10E94A92F680E791E1F5F1530E1
:1025100091F740904A0150904B0189EF681681E095
:10252000780634F081E090E09093EF058093EE051B
:102530008AEB97E040E855E260E070E00E943B31B2
:102540008AEB97E00E946C328823D1F387E691E012
:102550000E94860780EF95E00E94F12D80EF95E0C4
:102560000E94F92C85E592E00E94860780EF95E0B5
:102570006FE271E00E94ED2D8FE492E00E948607E9
:102580008DE392E00E94860780EF95E00E94B12DD6
:10259000682F8AEB97E040E150E00E94C63380EF5D
:1025A00095E00E94B12D882321F482E292E00E94FE
:1025B000860780913501882309F065C08091360136
:1025C000882309F060C080913701882309F05BC03F
:1025D00080913801882309F056C08091EE059091D2
:1025E000EF05892B21F487E092E00E94860700D056
:1025F0008DE391E0EDB7FEB79283818380EF95E0A4
:1026000060E671E040EC52E02FE231E000E510E0DE
:10261000B5E3EB2EB1E0FB2EA5E4CA2EA1E0DA2E45
:10262000F9E3AF2EF1E0BF2EE1E48E2EE1E09E2E25
:102630000E94062D0F900F902091EE053091EF052E
:10264000882339F0232BF9F481E092E00E94860779
:102650001AC0232B21F48BEE91E00E94860730EC08
:102660003093350128EA2093360191E090933701A9
:1026700089E1809338013093390120933A01909396
:102680003B0190933C012091490180EF95E06FE27E
:1026900071E045E351E030E00E94AB2D80EF95E022
:1026A00069E371E00E94962D8DED91E00E9486070E
:1026B0008091EC079091ED07009711F480EF97E07F
:1026C000BE016F5F7F4F681B790B8AEB97E04AE092
:1026D00050E00E9424348FEC91E00E9486070E9413
:1026E0005A07AB01BC018AEB97E02AE030E00E9478
:1026F000E43384EC91E00E948607B301882777FDDC
:102700008095982F920140E050E00E94BC3420E078
:1027100034E140E050E00E9402358AEB97E0BA01D4
:10272000A9012AE030E00E94A5338FEB91E00E94DE
:1027300086078091EE059091EF05892BE1F482EBFD
:1027400091E00E94860785E391E00E94050786EAF2
:1027500091E00E94860785E491E00E9405078AE9DE
:1027600091E00E94860789E391E00E9405078AEBC9
:1027700097E00E9405331092B5051092B4051092AF
:10278000B3051092B2051092E6051092E70510927B
:10279000E8051092E9051092E2051092E305109207
:1027A000E4051092E5051092DE051092DF05109207
:1027B000E0051092E1051092DA051092DB05109207
:1027C000DC051092DD050E94FD2E6093D20570930A
:1027D000D3058093D4059093D5056093CE0570936F
:1027E000CF058093D0059093D10581E090E00E94C1
:1027F0008B101092EB051092EA0580915C0190918C
:102800005D01892B09F055C080E090E020E030E0C8
:10281000F901E150FA4F11821082F901ED5EF94F92
:1028200011821082F901E95DF94F11821082F901DC
:10283000E55CF94F11821082F901E15BF94F1182D9
:102840001082F901ED59F94F11821082FC01E9580B
:10285000F94F1082FC01EF57F94F1082FC01E55748
:10286000F94F1082FC01EB56F94F1082FC01E15642
:10287000F94F1082FC01E755F94F1082FC01ED542D
:10288000F94F1082FC01E354F94F1082FC01E95327
:10289000F94F108201962E5F3F4F8A30910509F063
:1028A000B7CF1092ED051092EC051092B70510927B
:1028B000B60581E090E090935D0180935C010F90FC
:1028C0000F90CF91DF911F910F91FF90EF90DF90CC
:1028D000CF90BF90AF909F908F907F906F905F90C0
:1028E0004F9008955F926F927F928F929F92AF92D6
:1028F000BF92CF92DF92EF92FF920F931F93CF93ED
:10290000DF937C010E944F070E9432076C01F6940E
:10291000FE2CEE24F794E7948F2D8F708A3010F000
:10292000895C01C0805D80938004C701B4E0969506
:102930008795BA95E1F78870805D8093810480E384
:10294000809382048AE38093830480E280938404EA
:102950008701C5E0D0E0A0E8AA2EB12CAE0CBF1CC8
:10296000FDE05F2EEAE06E2E70E3772E6AE3862E9E
:1029700050E2952E84C0E016F1060CF057C0C80155
:102980008F709070892B09F051C0FE01E058FB4F09
:102990005082CE010196FC01E058FB4F60829C0101
:1029A0002F5F3F4F812F8F708A3010F0895C01C0FC
:1029B000805DF901E058FB4F80832F5F3F4FC801D6
:1029C000807F907044E0959587954A95E1F78A302D
:1029D00010F0895C01C0805DF901E058FB4F8083F5
:1029E000C9010196FC01E058FB4F70820196FC0181
:1029F000E058FB4F80820196FC01E058FB4F90822B
:102A0000EC012196C8018F739070892B79F4C0581E
:102A1000DB4F188280EF95E060E671E0A60120E8C8
:102A200034E00E949F2D6C01C0E0D0E088E197E087
:102A3000B8010E94F42D982F92959F70282F2F7027
:102A40009A3018F0892F895C02C0892F805DFE01C1
:102A5000E058FB4F8083CE0101962A3010F0295CAC
:102A600001C0205DFC01E058FB4F20830196FC0172
:102A7000E058FB4F9082EC0121960F5F1F4F0A1523
:102A80001B0509F078CFC058DB4F188280EF95E026
:102A900060E671E0A60120E834E00E949F2D0E94CC
:102AA0002807DF91CF911F910F91FF90EF90DF905A
:102AB000CF90BF90AF909F908F907F906F905F90DE
:102AC0000895CF92DF92EF92FF920F931F93CF93CF
:102AD000DF938C017B01EA01690188E197E06EE3F5
:102AE00070E043E50E94FB2D88E197E06FE370E022
:102AF00044E50E94FB2D88E197E060E470E042E449
:102B00000E94FB2D88E197E061E470E048E40E94B8
:102B1000FB2D88E197E062E470E0412F0E94FB2DDD
:102B200088E197E063E470E0402F0E94FB2D88E18C
:102B300097E064E470E043E50E94FB2D88E197E0B4
:102B400065E470E044E50E94FB2D88E197E066E4CF
:102B500070E042E40E94FB2D88E197E067E470E0BA
:102B60004CE40E94FB2D88E197E068E470E04F2D73
:102B70000E94FB2D88E197E069E470E04E2D0E94F1
:102B8000FB2D209709F45FC01C141D040CF05BC0E2
:102B9000CC16DD0608F057C088E197E06AE470E0E3
:102BA00043E50E94FB2D88E197E06BE470E04FE481
:102BB0000E94FB2D88E197E06CE470E043E40E9402
:102BC000FB2D88E197E06DE470E048E40E94FB2D66
:102BD00088E197E06EE470E04D2F0E94FB2D88E1C4
:102BE00097E06FE470E04C2F0E94FB2D88E197E0A6
:102BF00060E570E043E50E94FB2D88E197E061E528
:102C000070E04FE40E94FB2D88E197E062E570E000
:102C100043E40E94FB2D88E197E063E570E04CE41B
:102C20000E94FB2D4D2D552747FD5A9588E197E0D1
:102C300064E570E00E94FB2D88E197E065E570E0B7
:102C40004C2D0E94FB2DDF91CF911F910F91FF9092
:102C5000EF90DF90CF9008954F925F926F927F92A6
:102C60008F929F92AF92BF92CF92DF92EF92FF929C
:102C70000F931F93CF93DF933C0182E091E0B30168
:102C800044E050E00E947903009709F02FC1F3015E
:102C90001481C5E0D0E08824992454011CC0C501EA
:102CA000B4012AE030E040E050E00E94BC34212F23
:102CB000332727FD3095205330404901AA2497FC43
:102CC000A094BA2C860E971EA81EB91EF301EC0F15
:102CD000FD1F10812196812F80538A3018F4CA304D
:102CE000D105E9F6BE0161507040660D771D87E0A1
:102CF00091E044E050E00E947903009709F0F6C0AB
:102D0000F301EC0FFD1F53808E010C5F1F4FEF018D
:102D1000CC24DD2476011AC0C701B6012AE030E0D8
:102D200040E050E00E94BC34252D332727FD30952C
:102D3000205330406901EE24D7FCE094FE2CC60EEF
:102D4000D71EE81EF91E5B800F5F1F4F852D805335
:102D50008A3020F4219605311105F4F2B801615052
:102D60007040660D771D80E191E044E050E00E94E4
:102D70007903009709F07DC0A8014A5F5F4FF30116
:102D8000E00FF11F2381E8012496F301E00FF11F0A
:102D900000E010E014C0C801B3E0880F991FBA9595
:102DA000E1F7000F111F080F191F822F992787FDC8
:102DB0009095080F191F0053104023812196822FF0
:102DC00080538A3020F431964C175D0724F7280190
:102DD000BE0161507040660D771D85E191E044E0D1
:102DE00050E00E947903009719F020E030E02CC0F9
:102DF000DE011696F301EC0FFD1F6381AE014C5FFF
:102E00005F4FF301EC0FFD1F20E030E015C0C9015A
:102E100073E0880F991F7A95E1F7220F331F280F6F
:102E2000391F862F992787FD9095280F391F20532A
:102E3000304063814F5F5F4F862F80538A3020F48C
:102E40003196A417B5071CF70436110594F4201722
:102E500031077CF40333110564F0293231054CF05D
:102E6000109351010093500130935301209352016C
:102E700004C04424552420E030E0C814D904EA04F6
:102E8000FB04A0F5F8E38F16F1E39F06F0E0AF0630
:102E9000F0E0BF0658F181E488168AE6980680E0E3
:102EA000A80680E0B80610F5E0E7CE16E0E3DE06FF
:102EB000E0E0EE06E0E0FE06C8F0F1E9CF16F5E648
:102EC000DF06F0E0EF06F0E0FF0680F490924D019F
:102ED00080924C01D0924F01C0924E01C401B601C4
:102EE000A2010E946115C1E0D0E002C0C0E0D0E0C4
:102EF0000E944F070E943207AC01CD2B49F08FE4AE
:102F0000809380048BE680938104E2E0F0E00AC0C5
:102F100085E48093800482E7809381048093820417
:102F2000E3E0F0E0E058FB4F8AE08083118280EF1D
:102F300095E060E671E020E834E00E949F2D0E9459
:102F40002807DF91CF911F910F91FF90EF90DF90B5
:102F5000CF90BF90AF909F908F907F906F905F9039
:102F60004F900895EF92FF920F931F937C0108E119
:102F700017E0C80168E370E042E40E94FB2DC8013D
:102F800069E370E046E50E94FB2DC8016AE370E04A
:102F900049E40E94FB2DC8016BE370E04EE40E94FF
:102FA000FB2D4F2D552747FD5A95C8016CE370E066
:102FB0000E94FB2DC8016DE370E04E2D0E94FB2D99
:102FC0001F910F91FF90EF900895BF92CF92DF92E3
:102FD000EF92FF920F931F93CF93DF936C0182E0E8
:102FE00091E0B60144E050E00E947903009709F0B7
:102FF00049C0F601B480C5E0D0E0EE24FF2487018B
:103000001CC0C801B7012AE030E040E050E00E9457
:10301000BC342B2D332727FD3095205330407901C8
:103020000027F7FC0095102FE60EF71E081F191F4A
:10303000F601EC0FFD1FB08021968B2D80538A3056
:1030400018F4CA30D105E9F6D801C701815A9F406A
:10305000A040B04080569D46A040B04098F4F09209
:103060004B01E0924A012197CC0DDD1D8AE191E0F0
:10307000BE0145E050E00E947903009719F4C701B2
:103080000E94B21781E090E00E94E60BDF91CF91A1
:103090001F910F91FF90EF90DF90CF90BF90089518
:1030A0006F927F928F929F92AF92BF92CF92DF9258
:1030B000EF92FF920F931F93CF93DF936C01EB017D
:1030C000605A7E4F82E091E044E050E00E94790334
:1030D000009709F0D2C1CE0104960E941D05782EFA
:1030E00026E0E22EF12CEC0EFD1EC7010E941D050C
:1030F000682E80E2C816D10419F48824992419C0D6
:10310000CE0108960E941D05882E9AE0E92EF12C2A
:10311000EC0EFD1EC7010E941D05982EC114D1049E
:1031200051F096E2C916D10431F08FE2C816D104ED
:1031300011F0AA240BC082E090E0E80EF91EC7014E
:103140000E941D05A82EC114D10411F0BB2408C093
:1031500082E090E0E80EF91EC7010E941D05B82E1E
:103160008091B6059091B705892B09F443C08AEB8D
:1031700097E0672D4AE050E00E94B4338AEB97E075
:103180006EE20E94FD328AEB97E0662D4AE050E045
:103190000E94B4338AEB97E06EE20E94FD328AEB24
:1031A00097E0682D4AE050E00E94B4338AEB97E044
:1031B0006EE20E94FD328AEB97E0692D4AE050E012
:1031C0000E94B4338AEB97E06EE20E94FD328AEBF4
:1031D00097E06A2D4AE050E00E94B4338AEB97E012
:1031E0006EE20E94FD328AEB97E06B2D4AE050E0E0
:1031F0000E94C63398E0C916D10409F445C077206F
:1032000059F4662049F4882039F4992029F4AA2039
:1032100019F4BB2009F43DC188E1C816D10409F4B2
:1032200071C099E1C916D1046CF488E0C816D104C4
:1032300059F190E1C916D10409F445C0C114D10473
:1032400091F00FC086E2C816D10409F499C09FE23C
:10325000C916D10409F494C080E2C816D10409F457
:1032600070C0E601BDC088E197E060E070E04DE429
:103270000E94FB2D88E197E061E070E041E40E944C
:10328000FB2DC2E0D0E0ACC088E197E068E070E0E0
:1032900041E40E94FB2D88E197E069E070E044E49E
:1032A0000E94FB2D88E197E06AE070E044E40E9410
:1032B000FB2D88E197E06BE070E042E50E94FB2D7A
:1032C000CCE0D0E08DC088E197E060E170E04DE4B3
:1032D0000E94FB2D88E197E061E170E041E40E94EB
:1032E000FB2D88E197E062E170E043E50E94FB2D51
:1032F00088E197E063E170E04BE40E94FB2DC4E1BC
:10330000D0E06EC088E197E068E170E047E40E9499
:10331000FB2D88E197E069E170E041E40E94FB2D1C
:1033200088E197E06AE170E044E50E94FB2D88E1C6
:1033300097E06BE170E045E40E94FB2DCCE1D0E02A
:103340004FC088E197E060E270E040E50E94FB2D0D
:1033500088E197E061E270E04FE40E94FB2D88E194
:1033600097E062E270E042E50E94FB2D88E197E081
:1033700063E270E044E50E94FB2DC4E2D0E030C07F
:1033800086010F5F1F4F88E197E0B60141E40E947C
:10339000FB2D78010894E11CF11C88E197E0B8014D
:1033A00043E40E94FB2D87010F5F1F4F88E197E0E8
:1033B000B70143E40E94FB2DB8016F5F7F4F96E297
:1033C000C916D10431F4EB0188E197E0B80141E37B
:1033D00005C0EB0188E197E0B80142E30E94FB2DB4
:1033E0008E010F5F1F4F88E197E0BE01472D0E94BD
:1033F000FB2D78010894E11CF11C88E197E0B801ED
:10340000462D0E94FB2D80E2C816D10409F441C06C
:1034100087010F5F1F4F88E197E0B701482D0E9499
:10342000FB2D78010894E11CF11C88E197E0B801BC
:10343000492D0E94FB2DC114D10441F096E2C9161A
:10344000D10421F08FE2C816D10419F5E7012196C5
:1034500088E197E0B7014A2D0E94FB2DCD2811F09D
:103460007E0117C07E010894E11CF11C88E197E001
:10347000BE014B2D0E94FB2D0CC08091B605909192
:10348000B705892B21F081EC92E00E948607EE249B
:10349000FF24C701DF91CF911F910F91FF90EF9013
:1034A000DF90CF90BF90AF909F908F907F906F9064
:1034B0000895AF92BF92DF92EF92FF920F931F9306
:1034C000CF93DF93C091F105D091F205BE01605A10
:1034D0007E4FFB019E01AE01405C5F4F0AC09081B0
:1034E000892F81568A3110F4905290832F5F3F4F7D
:1034F00031962417350720F482E0213C380778F311
:1035000080E291E044E050E00E947903009781F06E
:103510000E944F07AC019093F2058093F10580EF74
:1035200095E060E671E02EE732E00E94A52D1FC213
:10353000CC59DE4F85E291E0BE0142E050E00E94AE
:103540007903009709F442C08091B6059091B705C0
:10355000892B21F083E792E00E9486078091F10594
:103560009091F2058B599E4F0E94D208EC018091F8
:10357000B6059091B705892B39F08AEB97E0BE012B
:103580004AE050E00E943734FE01B097E831F1057F
:1035900008F0F2C1EC5CFF4FEE0FFF1F0590F491B5
:1035A000E02D099420E030E08091B6059091B705B8
:1035B000892B11F421E030E03093B7052093B60554
:1035C000232B21F087E692E00E94860780E691E0B7
:1035D0000E94CF0ACCC16091F1057091F205675F3E
:1035E0007F4F80E090E023C06091F1057091F2057B
:1035F000675F7F4F88E090E01AC06091F10570919D
:10360000F205675F7F4F80E190E011C06091F105A6
:103610007091F205675F7F4F88E190E008C060918C
:10362000F1057091F205675F7F4F80E290E00E94A4
:103630005018A5C16091F1057091F205FB01E05AA7
:10364000FE4F8085813329F4675F7F4F86E290E0EB
:10365000EECF823309F093C1675F7F4F8FE290E036
:10366000E6CF80E090E00E94DF0A9093F20580931D
:10367000F10510925D0110925C0181C1C091F105CC
:10368000D091F205BE0167597E4F82E091E044E09F
:1036900050E00E947903009709F06EC1C05ADE4FD6
:1036A0006D85603319F480E090E004C0613341F52A
:1036B00081E090E00E948B1023C0C091F105D09171
:1036C000F205BE0164597E4F82E091E044E050E093
:1036D0000E9479030097A1F4C05ADE4F68896033D5
:1036E00029F410925F0110925E010AC0613311F05B
:1036F000623331F482E090E090935F0180935E0149
:1037000081E090E00E94DF0A32C181E090E002C0D7
:1037100080E090E00E94DF0A9093F2058093F1052B
:103720000E94FD2E6093C6057093C7058093C8055F
:103730009093C905A3C00091F1051091F205E8012D
:10374000C259DE4F82E091E0BE0144E050E00E94A9
:103750007903009709F042C01092C2051092C30588
:103760001092C4051092C505F801E05AFE4FD288A8
:10377000C3E1D0E0EE24FF2487015F011FC0C80130
:10378000B7012AE030E040E050E00E94BC342D2D2B
:1037900030E02053304079010027F7FC0095102FCE
:1037A000E60EF71E081F191FC731D10511F4DD24DD
:1037B00005C0F501EC0FFD1FD08021968D2D8053A3
:1037C0008A3018F4C831D105D0F2E092C205F092E7
:1037D000C3050093C4051093C5050FC088818032CE
:1037E00061F484E190E0A0E0B0E08093C2059093A2
:1037F000C305A093C405B093C5058091C2059091FF
:10380000C305A091C405B091C5054497A109B109AC
:103810008D569145A140B040E8F40E94422E20917F
:10382000C2053091C3054091C4055091C505260FCE
:10383000371F481F591F2093BE053093BF05409383
:10384000C0055093C10582E090E09093EB05809312
:10385000EA0508C01092C2051092C3051092C40573
:103860001092C5058091C2059091C3050E94800EFB
:103870009093F2058093F1050E94FD2E6093C2059E
:103880007093C3058093C4059093C50578C080915B
:10389000F1059091F20587599E4F61E070E008C0F4
:1038A0008091F1059091F20587599E4F60E070E09C
:1038B0000E94DC0E5CC00E94CD0D59C080E090E0FB
:1038C0000E94E60B54C08091F1059091F205855954
:1038D0009E4F0E94E5174BC0C091F105D091F205B3
:1038E000BE0165597E4F82E091E044E050E00E94C5
:1038F0007903009739F5FE01E05AFE4F6785FE0116
:10390000E059FE4F40E150E020E030E011C0C90135
:10391000A3E0880F991FAA95E1F7220F331F280F04
:10392000391F260F311D2053304061914F5F5F4F8B
:10393000862F80538A3018F44231510541F72031E7
:10394000310510F020E030E0C9010E9472140FC070
:1039500086E090E09093EB058093EA050DC080919E
:10396000F1059091F20584599E4F0E942C16909378
:10397000F2058093F10503C020E030E002C021E0B1
:1039800030E0C901DF91CF911F910F91FF90EF902F
:10399000DF90BF90AF9008952F923F924F925F9229
:1039A0006F927F928F929F92AF92BF92CF92DF924F
:1039B000EF92FF920F931F93CF93DF9376C4809182
:1039C000EA059091EB058330910509F47CC18430C0
:1039D000910534F4009781F0029709F00AC24AC1B8
:1039E0008530910509F4D8C1853091050CF4A6C144
:1039F000069709F0FEC113C180EF95E060EC72E01C
:103A000040E651E00E94FC2CAC0180EF95E060E6BE
:103A100071E00E94012D9093F2058093F105892BAE
:103A200009F463C08091B6059091B705892B89F19F
:103A300088E591E00E9486078AE190E01FC0E05A85
:103A4000FE4F8AEB97E060814AE050E00E94B43379
:103A50008091FD059091FE054D9728F48AEB97E043
:103A600060E071E004C08AEB97E068E271E00E94D8
:103A700056348091FD059091FE0501969093FE05C8
:103A80008093FD05E091FD05F091FE05EE31F10515
:103A9000B0F28AE190E00E949D07892B09F4A9C148
:103AA0000E94591A9093FC058093FB05892B09F01D
:103AB000A0C18091EA059091EB05892B09F099C18D
:103AC00080EF95E060E671E040E050E028EC30E007
:103AD0000E94A52D9093F2058093F10581E090E07E
:103AE0009093FC058093FB0584C180915E019091C9
:103AF0005F01039709F07DC12090D6053090D7056E
:103B00004090D8055090D90520E422162DE03206C9
:103B100023E0420620E0520638F400E1A02E07E23E
:103B2000B02EC12CD12C0CC0C201B10124E130E077
:103B300040E050E00E940235C901DA015C016D01EC
:103B40000E94FD2E2091CE053091CF054091D005E9
:103B50005091D105621B730B840B950BA616B7060B
:103B6000C806D90608F045C10E94FD2E7B018C01D4
:103B70006090D2057090D3058090D4059090D505C3
:103B8000E618F70808091909C201B1012CE030E074
:103B900040E050E00E9402352E153F0540075107D6
:103BA00008F027C18091CE059091CF05A091D00556
:103BB000B091D10586159705A805B90549F10E9470
:103BC000FD2E6093C2057093C3058093C405909346
:103BD000C50580EF95E00E94F62CAA0CBB1CCC1CFE
:103BE000DD1C8091D6059091D705A091D805B091A4
:103BF000D9058A199B09AC09BD098093540190939A
:103C00005501A0935601B093570185E090E056C04E
:103C100082E090E090935F0180935E01EAC00E9491
:103C2000FD2E6093C6057093C7058093C8059093D9
:103C3000C9052091C2053091C3054091C40550913A
:103C4000C505621B730B840B950B673971058105E4
:103C5000910508F4CEC081E090E00E94DF0A9093C5
:103C6000F2058093F10581E090E09093FC0580934C
:103C7000FB05BBC00E94FD2E2091C2053091C305FB
:103C80004091C4055091C505621B730B840B950BC5
:103C90006A3F71058105910508F4ABC081E090E0B1
:103CA0000E94DF0A9093F2058093F10581E090E095
:103CB0009093FC058093FB0583E090E09093EB05E7
:103CC0008093EA0596C00E94FD2E2091C205309196
:103CD000C3054091C4055091C505621B730B840B4D
:103CE000950B645F71408040904008F482C080EF83
:103CF00095E00E94F62C80915E0190915F01892BE6
:103D000031F082E090E090935F0180935E0184E067
:103D100090E09093EB058093EA0580E090E00E94AC
:103D20008B108091B6059091B705181619060CF006
:103D300060C088E491E00E9486075BC00E94422E2A
:103D40002091BE053091BF054091C0055091C1053D
:103D5000261737074807590708F04BC081E090E065
:103D60000E948B1080EF95E00E94F92C0E94FD2E9E
:103D70006093D2057093D3058093D4059093D505B5
:103D80008091B6059091B7051816190674F589E368
:103D900091E00E94860729C00E94FD2E2091C20555
:103DA0003091C3054091C4055091C505621B730B4A
:103DB000840B950B2091540130915501409156018F
:103DC00050915701621773078407950790F080EFB1
:103DD00095E00E94F92C0E94FD2E6093D20570930D
:103DE000D3058093D4059093D5051092EB051092DE
:103DF000EA050E94FD2E2091580130915901409111
:103E00005A0150915B01621B730B840B950B61533C
:103E100075478040904030F18091EA059091EB0524
:103E2000069701F180EA60E00E94CE0F1092B30580
:103E30001092B2050E94FD2E20E335E740E050E0ED
:103E40000E940235CA01B90120E335E740E050E0A5
:103E50000E94BC34609358017093590180935A01B9
:103E600090935B018091FB059091FC05019709F00F
:103E700045C10E94FD2E2091CE053091CF05409185
:103E8000D0055091D105621B730B840B950B6151CA
:103E900077428040904030F1C2EED5E009C0888181
:103EA0009981AA81BB818C839D83AE83BF83249734
:103EB00085E0C63DD80799F71092FE051092FD05E2
:103EC0000E94FD2E2091CE053091CF054091D00566
:103ED0005091D105621B730B840B950B6C837D8312
:103EE0008E839F830E94FD2E6093CE057093CF0535
:103EF0008093D0059093D10580915E0190915F01F0
:103F000002970CF4DEC06090DA057090DB058090BB
:103F1000DC059090DD05611471048104910409F4BD
:103F2000D0C02090DE053090DF054090E005509035
:103F3000E105211431044104510409F4C2C0209167
:103F4000E2053091E3054091E4055091E505211526
:103F500031054105510509F4B4C08091E605909101
:103F6000E705A091E805B091E9050097A105B10525
:103F700009F4A7C082017101E60CF71C081D191D88
:103F8000E20EF31E041F151FE80EF91E0A1F1B1F69
:103F9000B2E016950795F794E794BA95D1F7E092B9
:103FA000D605F092D7050093D8051093D905D8010E
:103FB000C701805C944DA140B04081549840AC460C
:103FC000B04008F07CC0C801B70124E130E040E017
:103FD00050E00E940235C901DA0157016801A81AB0
:103FE000B90ACA0ADB0A6A147B048C049D0408F42B
:103FF00066C09C01AD012E0D3F1D401F511F2615AF
:1040000037054805590508F45AC02A143B044C04E6
:104010005D0408F454C0221533054405550508F421
:104020004EC0E090E205F090E3050091E4051091A8
:10403000E505EA14FB040C051D0508F440C02E1527
:104040003F0540075107D8F1E090E605F090E705FD
:104050000091E8051091E905EA14FB040C051D0523
:1040600070F12E153F054007510748F180915E0120
:1040700090915F01029729F583E090E090935F01B2
:1040800080935E018091B6059091B705892BC9F0A8
:104090008FE291E00E9486074091D6055091D705A6
:1040A0006091D8057091D9058AEB97E02AE030E05D
:1040B0000E94A5338AE291E00E94860702C00E9416
:1040C000BB084091F1055091F20580EF95E060E664
:1040D00071E00E949A2DE0E6F1E080E090E002C0FD
:1040E0001192019622E0803C9207D0F39093FE0556
:1040F0008093FD051092FC051092FB050E94360985
:1041000090935F0180935E0182E00E945E30909305
:10411000FE058093FD054091F7055091F8056091EB
:10412000F9057091FA050097D9F44115510561051B
:10413000710559F40E94FD2E6093F7057093F80500
:104140008093F9059093FA05A9C00E94FD2E609313
:10415000F3057093F4058093F5059093F6059EC0E2
:10416000411551056105710509F459C08091F305A8
:104170009091F405A091F505B091F6050097A10581
:10418000B10509F44CC08E5E9240A040B040841B43
:10419000950BA60BB70B835E9440A040B04008F08F
:1041A0003EC060E070E08091B8059091B905892B20
:1041B00011F461E070E07093B9056093B80589E08F
:1041C0000E940A308091B8059091B9052091EE05C2
:1041D0003091EF05019789F4232B21F48DE191E0D3
:1041E0000E94860787E090E09093EB058093EA05B4
:1041F00080EF95E00E94F62C12C0232B21F484E17D
:1042000091E00E94860781E090E00E948B1080EF91
:1042100095E00E94F92C1092EB051092EA0510929D
:10422000F3051092F4051092F5051092F605109220
:10423000F7051092F8051092F9051092FA052EC0B4
:104240006091B2057091B305605E7B4F8AEB97E099
:1042500041E050E00E949834019749F48091B20502
:104260009091B30501969093B3058093B205809128
:10427000B2059091B305849731F4809143048F3750
:1042800011F40E9473058091B2059091B3058036B8
:10429000910524F01092B3051092B2058AEB97E0D5
:1042A0000E94C231181619065CF280915C0190914F
:1042B0005D01892B09F083CB0E945312DF91CF91CE
:1042C0001F910F91FF90EF90DF90CF90BF90AF9034
:1042D0009F908F907F906F905F904F903F902F9026
:1042E0000895EF92FF920F931F938091E30685301C
:1042F00011F5E090E806F090E9060091EA061091C9
:10430000EB068091E4069091E506A091E606B09157
:10431000E706E80EF91E0A1F1B1F0E94FD2EAA27A2
:1043200097FDA095BA2F8E159F05A007B10718F02D
:1043300086E08093E3068091E3061F910F91FF9042
:10434000EF90089585E08093E3060E94FD2EAA2752
:1043500097FDA095BA2F8093E4069093E506A0936D
:10436000E606B093E7060E941F2582E00895FF92BB
:104370000F931F93CF93DF938C01F62E1092EC06D0
:104380001092ED068091EE068F5F8093EE0680E935
:1043900091E0D801FC011D923197E9F76091EE069A
:1043A00070E0706E4091DE075091DF07C80124E491
:1043B00030E00E947328D80116962091EF063091C4
:1043C000F006C901FC0186E001900D928150E1F7F1
:1043D000C8016FEF70E046E050E00E94720382E88F
:1043E000D80151968C93519781E157968C938FEF1A
:1043F0009FEFAFEFBFEFF801868F978FA0A3B1A318
:1044000083E485A312A284E483A3BA9681E0D80151
:104410009A968C93818386E0828313828091DD0655
:104420009091DE06A091DF06B091E006848395832B
:10443000A683B7838091E1069091E20691878087F9
:10444000D801DA961D921D921D921C92DD977C96E2
:104450002091EF063091F006C901DC0186E00D9055
:1044600001928150E1F7D801AA5EBE4F93E6FD01AB
:10447000919382E811968C93DF01119683E58183F5
:10448000FD01319611969C93DF01119685E381839E
:10449000FD01319691E011969C93DF011196F18216
:1044A0009D012F5F3F4F8DE311968C93F90131965B
:1044B00087E0D90111968C939183EF012296409168
:1044C000EF065091F00620E030E0FE01E20FF31F0E
:1044D000DA01A20FB31F8C9180832F5F3F4F2630EC
:1044E000310599F78CE08E838AE08F83289620E04F
:1044F00030E0FE01E20FF31FD901A058BA4F8C91B2
:1045000080832F5F3F4F2A30310599F72A96D09349
:10451000F206C093F1062A97B3E0FB1609F042C0F9
:1045200082E38A8794E09B87E091DE07F091DF07C2
:1045300080818C87E091DE07F091DF0781818D8794
:10454000E091DE07F091DF0782818E87E091DE0740
:10455000F091DF0783818F8786E3888B998B629642
:10456000D093F206C093F1066297E091E007F091D4
:10457000E10780818A8BE091E007F091E10781817A
:104580008B8BE091E007F091E10782818C8BE091C9
:10459000E007F091E10783818D8B6696D093F20658
:1045A000C093F106A091F106B091F206FD0187E3F8
:1045B000819393E011969C93DF01119681E08183B2
:1045C0009D012F5F3F4F11969C93F901319686E034
:1045D000D90111968C938FEF81833296F093F20676
:1045E000E093F106E01BF10BBA97C801BF010E94EE
:1045F000D129DF91CF911F910F91FF90089563E032
:1046000070E00E94B72183E08093E3060895DF9273
:10461000EF92FF920F931F93CF93DF938C017B0157
:10462000E091DE07F091DF07EC018AAD9BADACAD08
:10463000BDAD80839183A283B383F801E65EFE4F14
:10464000E00EF11EDF011196D180ED0121968081EF
:104650008630C1F0873030F4813051F0833009F07A
:1046600057C00BC0833399F0863309F051C042C064
:10467000E091E407F091E50741C0E091E207F09195
:10468000E3073CC0E091DC07F091DD0737C01196ED
:104690006C9170E080E090E0982F872F762F66274E
:1046A0002981620F711D811D911D982F872F762FF3
:1046B00066272A81620F711D811D911D982F872FFA
:1046C000762F66272B81620F711D811D911D982FFA
:1046D000872F762F662728EE33E040E050E00E94D7
:1046E000BC346093E8067093E9068093EA069093E1
:1046F000EB060EC0E091E007F091E10711968D9175
:104700009D910D90BC91A02D80839183A283B38352
:10471000FE01ED0DF11DEE15FF0508F493CFC80164
:104720000E94FF2281E0DF91CF911F910F91FF90B6
:10473000EF90DF900895FC0166347105A0F183A12C
:10474000833489F5DF019A9682A5823061F514964B
:104750002D913D914D915C9117978091DD0690913F
:10476000DE06A091DF06B091E006281739074A0758
:104770005B07C9F4E65EFE4F8081EA51F140853364
:1047800091F4E45EFE4F8081EC51F140823019F0EB
:10479000853049F404C0CF010E9407230895CF015A
:1047A0000E94A221089580E00895CF92DF92EF92B7
:1047B000FF920F931F93CF93DF93EC017093F0065A
:1047C0006093EF065093DF074093DE073093E507D1
:1047D0002093E4071093E3070093E207F092E107C8
:1047E000E092E007D092DD07C092DC0780E090E025
:1047F0000E94A92F0E9450030E944B03AA2797FDF5
:10480000A095BA2F8F5D9C4BAA49BF4F8093DD06C0
:104810009093DE06A093DF06B093E0061092E206C6
:104820001092E10680E090E0E091DE07F091DF0772
:10483000E80FF91F1082E091E407F091E507E80F17
:10484000F91F1082E091E207F091E307E80FF91FEA
:104850001082E091E007F091E107E80FF91F108264
:10486000E091DC07F091DD07E80FF91F1082019657
:1048700084309105C9F6E091EF06F091F00685814C
:1048800082958F708F5B8093880585818F708F5B99
:10489000809389050E942825CE0161E070E00E9486
:1048A000B72181E08093E306DF91CF911F910F91B3
:1048B000FF90EF90DF90CF9008958AE061E00E9432
:1048C000CB2F8AE061E00E940A308BE061E00E9419
:1048D000CB2F8DE061E00E94CB2F8CE060E00E9446
:1048E000CB2F8BE061E00E940A308BE060E00E94F9
:1048F0000A308DE060E00E940A3081E58CBD8DB504
:1049000081608DBD08950F931F93CF93DF938C012A
:10491000EB01F89480918B0560E00E940A308AE7F1
:104920008EBD0DB407FEFDCF08C088818EBD0DB4CD
:1049300007FEFDCF21960150104001151105A9F782
:1049400080918B0561E00E940A307894DF91CF91CD
:104950001F910F9108950F931F93CF93DF93EC0155
:104960008B01F89480918B0560E00E940A308AE305
:104970008EBD0DB407FEFDCF09C01EBC0DB407FEF1
:10498000FDCF8EB5F80181938F0121972097A9F76C
:1049900080918B0561E00E940A307894DF91CF917D
:1049A0001F910F910895FF920F931F93082F162FB9
:1049B000F42EF89480918B0560E00E940A301F71FC
:1049C000102B1EBD0DB407FEFDCFFEBC0DB407FEBF
:1049D000FDCF80918B0561E00E940A3078941F9191
:1049E0000F91FF9008951F93182F282F30E0207605
:1049F00030708091F30690E02817390781F080EA43
:104A00006FE143E00E94D324412F40764093F306A8
:104A100042954695477080E86FE10E94D3241F912C
:104A200008950F931F93182F062F0E94F32480E4FC
:104A3000612F402F0E94D3241F910F910895609100
:104A4000F6066E7F6093F60688E30E9411250895AE
:104A50006091F60661606093F60688E30E94112576
:104A60000895682F677085E70E94112508950F93B8
:104A70001F93182F072F0E941125812F8F5F602F02
:104A80000E9411251F910F9108950F931F93182FC6
:104A9000062FF89480918B0560E00E940A30802FE9
:104AA0008F71812B8EBD0DB407FEFDCF1EBC0DB4E2
:104AB00007FEFDCF07FF04C01EBC0DB407FEFDCFEF
:104AC0001EB580918B0561E00E940A307894812F99
:104AD0001F910F9108951F93182F0E94F32480E0D7
:104AE000612F0E9445251F910895AF92BF92CF92EA
:104AF000DF92EF92FF920F931F93DF93CF9300D03B
:104B0000CDB7DEB76C015B0189E30E946B2588237A
:104B100019F400E010E051C06091F4067091F506C0
:104B200080E00E94372582E090E08E010F5F1F4FEA
:104B3000B8010E94AB2489819A819093F5068093F5
:104B4000F40682E090E0B8010E94AB24E980FA808C
:104B500082E090E0B8010E94AB24898187FD03C008
:104B600000E010E00DC0C70104978601015010401D
:104B70008017910708F48C01C801B5010E94AB248D
:104B80006091F4067091F5068CE00E9437256091E3
:104B9000F4067091F5066150704089E16F3F780727
:104BA00020F08CE06EEF79E101C08CE00E943725A7
:104BB00080E86EE140E40E94D324C8010F900F907A
:104BC000CF91DF911F910F91FF90EF90DF90CF90E9
:104BD000BF90AF90089582E70E946B25863008F061
:104BE0008F5F089580EA6EE140E20E94D3248DE158
:104BF0000E946B258823D9F380E86FE144E00E948E
:104C0000D324089580EA6FE144E00E94D3248DE12B
:104C10000E946B2582FDFBCF8FE10E946B2583FDF7
:104C2000FBCF80E86EE148E00E94D32480E86EE18B
:104C300040E20E94D32408950F931F93CF93DF93F4
:104C4000EC018B010FC08CE10E946B2581FF0AC033
:104C500080E86FE140E80E94D32480EA6FE140E8F9
:104C60000E94D32480E06FE10E94452583FDEBCFB5
:104C700082E06FEF79E10E943725BE016150764EE8
:104C800086E00E9437258AE760E040E00E94D32456
:104C9000CE01B8010E94832480E86FE148E00E94C1
:104CA000D324DF91CF911F910F9108950F931F93FC
:104CB000982F162F072F84ED692F0E94112586ED5E
:104CC000612F0E94112587ED602F0E94112504C0DD
:104CD0008FE090E00E94642F8AEE0E946B2580FD99
:104CE000F7CF1F910F9108950F931F938C01862F7B
:104CF00060938B0561E00E94CB2F80918B0561E072
:104D00000E940A3078948FEF60E04FEF0E94D32426
:104D100062E370E080E090E00E940B2F1092F506B5
:104D20001092F40688E060E070E00E9437258CE085
:104D300060E070E00E9437258AE06EEF79E10E9422
:104D4000372584E06FEF79E10E94372586E06FEF29
:104D50007FE10E94372581EB8093F60688E361EBC3
:104D60000E94112588E26FE370E30E94372580E3FB
:104D700069EF77EF0E94372580EC6DE00E941125E6
:104D800081EC60E00E94112580E862EC42E30E9421
:104D9000D32486EC62E17CE00E94372584EC62E15A
:104DA0000E9411258AEC6CED75E00E94372584EE97
:104DB000F80160810E94112585EEF80161810E9451
:104DC000112582EEF80162810E94112583EEF8011F
:104DD00063810E94112580EEF80164810E941125F3
:104DE00081EEF80165810E94112580E160E071E0AB
:104DF0000E9456268FE10E94F32480E86BE140EC8C
:104E00000E94D32480E86FE144E00E94D3241F91E4
:104E10000F910895682F84ED0E94112582ED61E0C5
:104E20000E9411258FE090E00E94642F8AEE0E947C
:104E30006B2580FDFBCF82ED60E00E94112589ED9E
:104E40000E946B2590E0089581E10E940A2720E0EE
:104E5000892B09F021E0822F0895CF92DF92EF9203
:104E6000FF920F931F93CF93DF936C01413081F436
:104E7000685070407B0100E010E0685F7F4F21E1E7
:104E800030E040E050E0E20EF31E041F151F15C095
:104E9000423021F0EE24FF2487010FC0685070409B
:104EA0007B0100E010E0685F7F4F86E090E0A0E0CB
:104EB000B0E0E80EF91E0A1F1B1FF601EB0116C039
:104EC000808190E0A0E0B0E0BA2FA92F982F88272A
:104ED000218130E040E050E0822B932BA42BB52BB6
:104EE000E80EF91E0A1F1B1F32962297C230D10509
:104EF00038F7FB01EE7FEC0DFD1D60FF15C08081D2
:104F000090E0A0E0B0E0BA2FA92F982F882708C022
:104F10002FEF3FEF40E050E0E222F322042315237D
:104F2000E80EF91E0A1F1B1FC801AA27BB270097FE
:104F3000A105B10569F7970120953095C901DF9169
:104F4000CF911F910F91FF90EF90DF90CF90089538
:104F5000CF93DF93EC015093FD064093900520E042
:104F600030E0F901EC5EF84FDB01A20FB31F8C912A
:104F700080832F5F3F4F2430310599F720E030E0E8
:104F8000F901EA51F84FDE01A20FB31F8C91808323
:104F90002F5F3F4F2630310599F7DF91CF9108956C
:104FA000FC0169327105B0F08485883099F48585FB
:104FB000863081F4DF019696E4E1F7E09C918081F0
:104FC000981741F41196319687E0E831F807B1F768
:104FD00081E0089580E00895FC016A327105D0F007
:104FE00084858830B9F485858823A1F48685853445
:104FF00089F4DF01E4E1F7E05E969C915E978081A1
:10500000981741F41196319687E0E831F807A1F737
:1050100081E0089580E008950F931F938C01FC01B7
:10502000108E118E80E4848B158A868BC8010E96B3
:1050300064E170E040E00E942D27F801908F818F9D
:105040001F910F910895AC01FC01A4E1B7E0828D9E
:10505000868F8D91828F319687E0A831B807B9F796
:10506000CA010E940C280895FC01B99694E0808141
:10507000680F711D84816483442311F0808301C013
:10508000108291503197992319F0672F7727EFCF2E
:1050900008950F931F938C01FC0194A182A184A316
:1050A00092A395A183A185A393A3C8010E9434284C
:1050B000F80112AA13AA80E586A71F910F910895FF
:1050C0006A5C7F4FDC01A60FB71F6653704003C0B8
:1050D0008D936F5F7F4FFA014F5F5F4F84918823FD
:1050E000B9F7CB010895FF920F931F93CF93DF93EE
:1050F000EC01F62E072FBA01122F932FAE019E015D
:10510000A0E0B0E0FD01E65FF84F8081F901808307
:10511000FD01EA51F84F8081F901868311962F5FD6
:105120003F4FA630B10571F788E08C871D86DE0100
:10513000E6E3F4E084911E968C931E9731961196C7
:1051400084E0EF33F807B1F7188A81E18F8BA0E094
:10515000B0E0FB01EA0FFB1F8081FA01868FFD01A1
:10516000EC5EF84F8081FA01828F11964F5F5F4F9E
:10517000A430B10571F79CA31DA30AA3FBA21EA234
:1051800018A619A6DF91CF911F910F91FF90089556
:10519000AC0181E080938C0520E030E0F901EA5F0A
:1051A000F84FDA01A20FB31F8C9180832F5F3F4F1E
:1051B0002430310599F70895CF93DF93EB01BA01BD
:1051C000DA010D900020E9F71197A41BB50BE696C4
:1051D000AC014C0F5D1FE6979D0108C0FB0181915A
:1051E000BF01FA018193AF012150304021153105F3
:1051F000A9F79E012A0F3B1FC901DF91CF910895A6
:10520000FF920F931F93CF93DF93EC01F62E142F91
:10521000022FAC01DC0120E030E0F901E65FF84F3D
:1052200080818C93F901EA51F84F808116968C9316
:1052300016972F5F3F4F11962630310571F788E0A2
:105240008C871D86DE01E6E3F4E084911E968C9344
:105250001E973196119684E0EF33F807B1F78CE290
:10526000898B86E08F8B20E030E0F901E05FF84F1A
:105270008081FA01868FF901EC5EF84F8081FA0196
:10528000828F2F5F3F4F4F5F5F4F2430310569F7AB
:10529000CE010E940C281CA30DA38BE08AA3FBA2C5
:1052A000FE01B69680E011928F5F8830E1F7809121
:1052B000910588A78D5F8093910580E68EA782E097
:1052C0008FA794E098AB19AA1AAA1BAA1CAA1DAA18
:1052D0008EAB9FAB88AF86E289AFCE014A9660E283
:1052E00070E042E00E942D279AAB8BAB8AE390E0FE
:1052F000BE010E941C26DF91CF911F910F91FF905C
:105300000895CF93DF93EC01AC0126EE37E0FC016A
:10531000D9019FEF90838D918683319687E0AC3ED3
:10532000B807C1F788E08C8786E08D87DE01EEE262
:10533000F4E084911E968C931E973196119684E02A
:10534000E633F807B1F7F90181919F01FA01868BE5
:1053500010A24F5F5F4FF7E02C3E3F07A1F7DE0141
:105360005C9620E030E0FB01E20FF31F80811A968B
:105370008C931A97F901EC5EF84F80818D932F5F23
:105380003F4F2430310579F780918C0588608093F8
:105390008C058AE290E0BE010E941C26DF91CF912D
:1053A0000895DF92EF92FF920F931F938C017B0180
:1053B0008CE190E0E80EF91EF801F08A84EE9FEF90
:1053C000E80EF91EDE2C9CE1D90ED18AC8010E949C
:1053D0000C28E8E0F0E0EE0EFF1EF801F6A2FCEE6D
:1053E000DF0EF801D7A288E090E0E80EF91EC801B0
:1053F0004A96B70141E00E942D27F80190A781A7A6
:10540000C7014A96B8010E941C261F910F91FF9078
:10541000EF90DF900895EF92FF920F931F938C010E
:105420007B01CB018896F801908B818BC8010E948B
:105430000C28F80112AA13AA8CE190E0E80EF91EDC
:10544000C8014A96B70142E00E942D27F80192ABAD
:1054500083ABC7014A96B8010E941C261F910F9189
:10546000FF90EF900895CF93DF93EC01FC01A6EE3F
:10547000B7E0868180838D918683319687E0AC3E4C
:10548000B807B9F7842F80618FA7443029F06115E0
:10549000710511F461E070E0CE0141E00E944928FD
:1054A000188A88E2898BCE010E94232884E088AB89
:1054B00019AACE014A966CE170E042E00E942D27C5
:1054C0009AAB8BAB86E390E0BE010E941C26DF9175
:1054D000CF910895EF92FF920F931F938C017B0160
:1054E0006091FE067091FF0640E00E94332A89E138
:1054F000F80187A7C801B7010E940B2A1F910F91DD
:10550000FF90EF900895CF93DF93EC01FC01A6EE9E
:10551000B7E0868180838D918683319687E0AC3EAB
:10552000B807B9F7188A8CE2898BCE010E9423282C
:1055300082E18FA7CE0161E070E040E00E9449283F
:105540001EA21FA28091910588A719A68D5F809346
:10555000910582E08EAB84E08FAB95E098AF19AEF9
:1055600080E68EA798AB88E789ABCE014A9660E2C9
:1055700070E042E00E942D279AAB8BAB8AE390E06B
:10558000BE010E941C26DF91CF9108950F931F93B7
:10559000CF93DF93EC018B01FC01A6EEB7E086818F
:1055A00080838D918683319687E0AC3EB807B9F74A
:1055B000CE010E9423281AA28CA1883F18F08DA149
:1055C0008F5F8DA38CA1885F8CA3C801BE010E9450
:1055D0001C26DF91CF911F910F910895CF93DF93F8
:1055E000AC01EC0126EE37E0FC01D9018681808315
:1055F0008D918683319687E0AC3EB807B9F7FA0102
:10560000148A82E0858B8E8988A3F90181919F019C
:105610008E8B2196F7E02C3E3F07A9F7FA017C9686
:10562000A4E1B7E0808182878D91819387E0A831E2
:10563000B807C1F78AE290E0BA010E941C26DF9108
:10564000CF910895EF92FF920F931F93CF93DF9323
:10565000EC017B016115710509F040C080918C055A
:1056600080FD04C080918C0582FF0FC080918D0564
:1056700090918E05892B49F40E942427882329F0D4
:10568000CE0166E077E00E94812980918D0590919E
:105690008E05019690938E0580938D058091F70677
:1056A000813009F08FC180918C0581FF8BC182E030
:1056B0008093F70680918F058F5F80938F058F71A0
:1056C0006091F8066295660F607E682BCE0140916E
:1056D000F9062091FA060E94002974C10E94D02781
:1056E000882341F18D89813019F4CE010E94EE2A80
:1056F00080918C0583FF66C18D89823009F062C17B
:10570000E6E0F7E0DE015C969C915C97808198175B
:1057100009F058C11196319687E0EA30F80799F7F9
:10572000EAE0F7E08E898193219697E0E031F9076E
:10573000C9F752C1CE01B7010E94EC27882309F4B2
:1057400041C19F89913149F48AA18823C9F48BA171
:105750008533B1F46AE270E037C1913089F48AA1EF
:10576000883071F4E0910407F0910507309719F043
:10577000CE014A960995CE01B7010E94C62A22C1E0
:1057800086E3E816F10418F4963009F01BC19CA1D9
:105790009B3009F0C9C0D093FC06C093FB06DE0124
:1057A000E0E1F7E05A969C915A978081981709F0AA
:1057B00009C11196319697E0E431F90799F710C1C4
:1057C000E0910007F0910107309709F4A3C08DA183
:1057D00082958695877063E040E050E020E030E0FD
:1057E000099598C0988980E02989022F10E0082B3C
:1057F000192B8EA582958F70482F50E0CA01880F13
:10580000991F880F991F081B190B0451104017FF8F
:1058100002C000E010E0B8018091F706823089F5FF
:1058200031FF20C034FF1EC0CE0160E070E040E0D8
:105830000E94332A88E18FA7E0910207F0910307C5
:10584000309719F460E070E006C08BA182958695D0
:1058500087700995BC0183E08093F706CE010E9412
:105860000B2AB0C081E08093F7068FA584FF03C0A8
:1058700060E070E003C0B8016F5F7F4FCE0144E08D
:105880008CC0843039F4E0910007F0910107309723
:1058900089F432C0833099F584E08093F706E09173
:1058A0000007F0910107309739F18EA582958F702E
:1058B000482F50E0440F551F440F551FC70108974C
:1058C0004E5D5F4F8417950708F4AC01C801840F43
:1058D000951FE816F90610F0980103C09701241BE4
:1058E000350B8DA182958695877060E00995882398
:1058F00019F0CE01B8010BC0CE01B8014DC0853002
:1059000009F460C030FF0AC06F5F7F4FCE0149E0ED
:105910000E94332A85E08093F70654C001151105D3
:1059200009F452C0CE0138C08091FD06981709F0E5
:1059300049C09DA180919005981709F043C08FA59B
:1059400081FF04C0CE010E94832A3CC084FF3AC07C
:10595000988980E02989422F50E0482B592B2EA5A9
:10596000822F82958F7090E0880F991F880F991F62
:10597000481B590B4451504057FF02C040E050E0D3
:105980005093FF064093FE06452B51F48FA580FFF0
:1059900019C0CE0160E070E040E00E94332A12C0DE
:1059A0008EA582958F70682F70E0660F771F660F47
:1059B000771F6E5D7F4F88EF9FEFE80EF91EE616AA
:1059C000F70610F460E070E0CB01DF91CF911F91FA
:1059D0000F91FF90EF90089582E080938C05F2CFB5
:1059E0008FA5382F82FDECCEFDCE08950E940226B1
:1059F00008950E94F2250895CB01BA010E947525F1
:105A00000895CB01BA010E94222B08952F923F9254
:105A10005F926F927F928F929F92AF92BF92CF923E
:105A2000DF92EF92FF920F931F93DF93CF93CDB747
:105A3000DEB72A970FB6F894DEBF0FBECDBF3B018D
:105A40005A8349833C832B83FE82ED82D886CF82A2
:105A5000BA86A98614010E94FD2EAC01CB01DA01A1
:105A60004C015D01C3016B817C814D815E812F8181
:105A7000388509851A857101CE8CDF8C0E94D5236B
:105A800088E0582E89819A81B3010E9475258C0186
:105A9000C301B8010E94222B892BA1F7C301B801D1
:105AA0000E949B230E947121853011F481E026C061
:105AB0000E94FD2EA50194012059384E4F4F5F4F93
:105AC0002617370748075907E8F60E94FD2E5A9413
:105AD000A1F0AC01CB01DA014C015D01C3016B8186
:105AE0007C814D815E812F81388509851A85710100
:105AF000CE8CDF8C0E94D523C5CF80E02A960FB6CE
:105B0000F894DEBF0FBECDBFCF91DF911F910F91F3
:105B1000FF90EF90DF90CF90BF90AF909F908F90CD
:105B20007F906F905F903F902F900895CB010E94DF
:105B3000C8280895CB01BA010E946A2A0895CB01B2
:105B4000BA01A9010E94DC280895CB01BA01A9017C
:105B50000E9460280895CB01BA01A9010E94A827DC
:105B600008950E94EB250895CF93DF93CB01642F16
:105B70000E94742682E00E9431256AE070E080E095
:105B800090E00E940B2FC0E0D0E084E160E878E371
:105B90000E94562664EF71E080E090E00E940B2F97
:105BA00084E160E979E30E94562664EF71E080E0C9
:105BB00090E00E940B2F2196C330D10531F784E18C
:105BC00066E774E30E94562664E670E080E090E0A9
:105BD0000E940B2FDF91CF9108954AE00E94B42DCF
:105BE00008950E945D240895F999FECF72BD61BDAC
:105BF000F89A80B50895F999FECF1FBA72BD61BDBC
:105C000040BD0FB6F894FA9AF99A0FBE08958091A4
:105C1000230790912407089560939205709393054C
:105C20008093940590939505089560931B07709356
:105C30001C0780931D0790931E07209192053091B9
:105C400093054091940550919505260F371F481FE5
:105C5000591F20931F07309320074093210750932B
:105C6000220782E090E090932407809323070E940C
:105C7000FD2E609325077093260780932707909346
:105C800028070895EF92FF920F931F931CC02F5F78
:105C90003F4F4F4F5F4F20931B0730931C0740939C
:105CA0001D0750931E0788EE93E0A0E0B0E0E80ED9
:105CB000F91E0A1F1B1FE0922507F092260700938A
:105CC0002707109328070E94FD2EE0902507F090EB
:105CD000260700912707109128076E197F09800B6E
:105CE000910B20911B0730911C0740911D0750918B
:105CF0001E07685E73408040904048F680911F0701
:105D000090912007A0912107B09122072817390709
:105D10004A075B07E8F0E0911907F0911A073097FE
:105D200049F00995611571058105910519F00E94E9
:105D3000152E0EC020E030E08091230790912407BB
:105D4000892B11F021E030E03093240720932307C2
:105D500060911B0770911C0780911D0790911E0791
:105D60001F910F91FF90EF9008951F920F920FB621
:105D70000F9211242F933F938F939F93AF93BF93D1
:105D800080912D0790912E07A0912F07B091300799
:105D9000309131070196A11DB11D232F2D5F2D37A5
:105DA00020F02D570196A11DB11D2093310780933E
:105DB0002D0790932E07A0932F07B0933007809163
:105DC000290790912A07A0912B07B0912C070196E3
:105DD000A11DB11D8093290790932A07A0932B073B
:105DE000B0932C07BF91AF919F918F913F912F91CD
:105DF0000F900FBE0F901F9018958FB7F8942091B9
:105E00002D0730912E0740912F07509130078FBFFB
:105E1000B901CA0108959B01AC017FB7F894809144
:105E2000290790912A07A0912B07B0912C0766B5FE
:105E3000A89B05C06F3F19F00196A11DB11D7FBF42
:105E4000BA2FA92F982F8827860F911DA11DB11D4C
:105E500062E0880F991FAA1FBB1F6A95D1F7BC018A
:105E60002DC0FFB7F8948091290790912A07A0913F
:105E70002B07B0912C07E6B5A89B05C0EF3F19F0A2
:105E80000196A11DB11DFFBFBA2FA92F982F8827FA
:105E90008E0F911DA11DB11DE2E0880F991FAA1F51
:105EA000BB1FEA95D1F7861B970B885E9340C8F21B
:105EB000215030404040504068517C4F2115310501
:105EC0004105510571F60895019739F0880F991F22
:105ED000880F991F02970197F1F70895789484B578
:105EE000826084BD84B5816084BD85B5826085BDD6
:105EF00085B5816085BDEEE6F0E0808181608083BC
:105F0000E1E8F0E01082808182608083808181609E
:105F10008083E0E8F0E0808181608083E1EBF0E065
:105F2000808184608083E0EBF0E080818160808309
:105F3000EAE7F0E0808184608083808182608083F2
:105F40008081816080838081806880831092C1001D
:105F50000895982F8E3008F09E5097708091960586
:105F60008295880F880F807C892B80937C0080919C
:105F70007A00806480937A0080917A0086FDFCCF5D
:105F80002091780040917900942F80E030E0282B18
:105F9000392BC9010895CF93DF93482F50E0CA01F0
:105FA0008C589A4FFC013491405A5A4FFA0184910F
:105FB000882369F190E0880F991FFC01EE5BFA4F8E
:105FC000A591B491FC01E45BFA4FC591D49166238D
:105FD00051F42FB7F8948C91932F909589238C933B
:105FE000888189230BC0623061F42FB7F8948C91BB
:105FF000932F909589238C938881832B88832FBF3F
:1060000006C09FB7F8948C91832B8C939FBFDF9130
:10601000CF910895482F50E0CA0188579A4FFC014C
:106020002491CA018C589A4FFC019491405A5A4FBE
:10603000FA013491332309F440C0222351F1233073
:1060400071F0243028F42130A1F0223011F514C071
:106050002630B1F02730C1F02430D9F404C080914B
:1060600080008F7703C0809180008F7D80938000B7
:1060700010C084B58F7702C084B58F7D84BD09C000
:106080008091B0008F7703C08091B0008F7D8093A6
:10609000B000E32FF0E0EE0FFF1FE45BFA4FA59195
:1060A000B4912FB7F894662321F48C9190958923AD
:1060B00002C08C91892B8C932FBF0895682F70E0BC
:1060C000CB0188579A4FFC012491CB018C589A4FF1
:1060D000FC014491605A7A4FFB019491992319F481
:1060E00020E030E03CC0222351F1233071F0243015
:1060F00028F42130A1F0223011F514C02630B1F07F
:106100002730C1F02430D9F404C0809180008F770B
:1061100003C0809180008F7D8093800010C084B583
:106120008F7702C084B58F7D84BD09C08091B00097
:106130008F7703C08091B0008F7D8093B000892F4E
:1061400090E0880F991F8A5A9A4FFC01A591B4914B
:106150008C9120E030E0842311F021E030E0C9018F
:10616000089508951F920F920FB60F9211242F9346
:106170003F934F938F939F93EF93FF938091C00032
:1061800082FD1DC04091C6002091720730917307B7
:106190002F5F3F4F2F733070809174079091750778
:1061A0002817390771F0E0917207F0917307EE5CE0
:1061B000F84F4083309373072093720702C0809199
:1061C000C600FF91EF919F918F914F913F912F9139
:1061D0000F900FBE0F901F901895E091C607F09199
:1061E000C707E05CFF4F8191919120813181821B33
:1061F000930B8F739070892B11F00E94B13008952A
:106200001F920F920FB60F9211242F933F938F93EB
:106210009F93EF93FF932091B6073091B70780913A
:10622000B8079091B9072817390731F48091C10058
:106230008F7D8093C10014C0E091B807F091B90739
:10624000EA58F84F20818091B8079091B9070196DC
:106250008F7390709093B9078093B8072093C6000E
:10626000FF91EF919F918F913F912F910F900FBED2
:106270000F901F901895AF92BF92DF92EF92FF920E
:106280000F931F93CF93DF93EC017A018B01DD24F1
:10629000403081EE580780E0680780E0780711F011
:1062A000DD24D39491E0A92EB12CEC89FD89DD2069
:1062B00069F0C50108A002C0880F991F0A94E2F78F
:1062C000808360E079E08DE390E005C0108260E8B3
:1062D00074E88EE190E0A80197010E9402352150F8
:1062E000304040405040569547953795279580E17E
:1062F0002030380720F0DD2011F0DD24D6CFE889EA
:10630000F9893083EA89FB89208319A2EE89FF8904
:10631000408121E030E0C9010C8C02C0880F991F38
:106320000A94E2F7482B4083EE89FF894081C90136
:106330000D8C02C0880F991F0A94E2F7482B408306
:10634000EE89FF894081C9010E8C02C0880F991F18
:106350000A94E2F7482B4083EE89FF8980810F8CF5
:1063600002C0220F331F0A94E2F7209528232083CE
:10637000DF91CF911F910F91FF90EF90DF90BF9031
:10638000AF900895DC011C96ED91FC911D97E05CA7
:10639000FF4F2191319180819181281B390B2F73FF
:1063A0003070C9010895DC011C96ED91FC911D9798
:1063B000E05CFF4F20813181E054F040DF01AE5BB3
:1063C000BF4F8D919C9111972817390719F42FEF22
:1063D0003FEF07C08D919C91E80FF91F8081282F16
:1063E00030E0C9010895DC011C96ED91FC911D97E8
:1063F000E05CFF4F20813181E054F040DF01AE5B73
:10640000BF4F8D919C9111972817390719F42FEFE1
:106410003FEF10C08D919C911197E80FF91F2081DB
:106420008D919C91119701968F73907011969C930A
:106430008E9330E0C9010895DC0191968C9191977B
:10644000882339F05496ED91FC915597808186FF11
:10645000F9CF91961C920895CF93DF93EC01EE85CE
:10646000FF85E05CFF4F20813181E054F0402F5FD9
:106470003F4F2F733070DF01AE5BBF4F8D919C910A
:10648000119728173907D1F3E05CFF4F8081918184
:10649000E054F040E80FF91F6083EE85FF85E05C73
:1064A000FF4F31832083EE89FF89208181E090E0D6
:1064B0000F8C02C0880F991F0A94E2F7282B2083C3
:1064C00081E089A3EC89FD8980818064808381E0FB
:1064D00090E0DF91CF91089581E008951092BD077B
:1064E0001092BC0788EE93E0A0E0B0E08093BE0776
:1064F0009093BF07A093C007B093C1078BE995E0C5
:106500009093BB078093BA0782E397E09093C70705
:106510008093C60786E797E09093C9078093C807E2
:1065200085EC90E09093CB078093CA0784EC90E0D1
:106530009093CD078093CC0780EC90E09093CF07A9
:106540008093CE0781EC90E09093D1078093D007A1
:1065500082EC90E09093D3078093D20786EC90E092
:106560009093D5078093D40784E08093D60783E087
:106570008093D70787E08093D80785E08093D90779
:1065800081E08093DA070895CF93DF930E946E2F06
:106590000E945312CDEED0E30E94CC1C2097E1F371
:1065A0000E94ED30F9CFCF92DF92EF92FF920F93DE
:1065B0001F93CF93DF937C016B018A01C0E0D0E091
:1065C0000FC0D6016D916D01D701ED91FC91019045
:1065D000F081E02DC7010995C80FD91F0150104067
:1065E0000115110571F7CE01DF91CF911F910F9128
:1065F000FF90EF90DF90CF900895DC01ED91FC913A
:106600000190F081E02D09950895EF92FF920F938C
:106610001F938C01DC01ED91FC910190F081E02D44
:106620006DE009957C01D801ED91FC910190F0811C
:10663000E02DC8016AE009959C012E0D3F1DC9019E
:106640001F910F91FF90EF900895CF93DF93EC018E
:106650006115710519F420E030E00FC0DB010D90E9
:106660000020E9F71197A61BB70BE881F98102809A
:10667000F381E02DAD0109959C01C901DF91CF9116
:1066800008954F925F927F928F929F92AF92BF92A6
:10669000CF92DF92EF92FF920F931F93DF93CF93EE
:1066A000CDB7DEB7A1970FB6F894DEBF0FBECDBF52
:1066B0002C01742ECB01223008F42AE019A231E219
:1066C000C32ED12CCC0EDD1E822E9924AA24BB24ED
:1066D000672D752FA50194010E94023579018A0169
:1066E000C801B701A50194010E94BC34472D461B87
:1066F0000894C108D1084A3014F4405D01C0495CD7
:10670000F6014083E114F1040105110521F07E2C0E
:106710005F2DC801DDCFC201B6010E942533A196CD
:106720000FB6F894DEBF0FBECDBFCF91DF911F91A2
:106730000F91FF90EF90DF90CF90BF90AF909F9020
:106740008F907F905F904F900895DC012115310567
:1067500041F4ED91FC910190F081E02D642F0995B9
:1067600008950E9441330895EF92FF920F931F9373
:106770009A01E62EFF2400E010E0B801A7010E9474
:10678000A5331F910F91FF90EF900895CF92DF9264
:10679000EF92FF920F931F936C01E62E9A01FF2454
:1067A00000E010E0B801A7010E94A5338C01C601EA
:1067B0000E940533080F191FC8011F910F91FF9008
:1067C000EF90DF90CF900895CF92DF92EF92FF92FB
:1067D0000F931F93CF93DF93EC016A017B01211587
:1067E000310541F4E881F9810190F081E02D642FB9
:1067F00009951FC02A303105D1F477FF17C0E88111
:10680000F9810190F081E02D6DE209958C0144271A
:106810005527BA014C195D096E097F09CE012AE09E
:106820000E9441339801280F391F04C02AE00E94BA
:1068300041339C01C901DF91CF911F910F91FF90CE
:10684000EF90DF90CF900895EF92FF920F931F93F8
:106850007B019A010027F7FC0095102FB801A701D2
:106860000E94E4331F910F91FF90EF900895CF9213
:10687000DF92EF92FF920F931F936C017B019A01BD
:106880000027F7FC0095102FB801A7010E94E43300
:106890008C01C6010E940533080F191FC8011F9102
:1068A0000F91FF90EF90DF90CF9008950E942533D5
:1068B0000895EF92FF920F931F937C010E9425335E
:1068C0008C01C7010E940533080F191FC8011F91D1
:1068D0000F91FF90EF900895CF93DF93EC010E940A
:1068E000FD2E688779878A879B87E881F9810680F2
:1068F000F781E02DCE0109959C0197FF15C00E94FC
:10690000FD2E288539854A855B85621B730B840BB8
:10691000950B2C813D814E815F816217730784073F
:10692000950718F32FEF3FEFC901DF91CF9108953D
:10693000CF92DF92EF92FF920F931F93CF93DF934B
:106940006C018B017A01C0E0D0E009C0C6010E9451
:106950006C3497FD07C0F80181938F012196CE1505
:10696000DF05A0F3CE01DF91CF911F910F91FF9032
:10697000EF90DF90CF900895629FD001739FF00158
:10698000829FE00DF11D649FE00DF11D929FF00DBF
:10699000839FF00D749FF00D659FF00D9927729FF6
:1069A000B00DE11DF91F639FB00DE11DF91FBD0181
:1069B000CF0111240895AA1BBB1B51E107C0AA1FD8
:1069C000BB1FA617B70710F0A61BB70B881F991F90
:1069D0005A95A9F780959095BC01CD01089597FB34
:1069E000092E07260AD077FD04D0E5DF06D0002067
:1069F0001AF4709561957F4F0895F6F790958195FB
:106A00009F4F0895A1E21A2EAA1BBB1BFD010DC0CA
:106A1000AA1FBB1FEE1FFF1FA217B307E407F5074E
:106A200020F0A21BB30BE40BF50B661F771F881F2A
:106A3000991F1A9469F760957095809590959B01C0
:106A4000AC01BD01CF01089597FB092E05260ED09C
:106A500057FD04D0D7DF0AD0001C38F4509540957C
:106A6000309521953F4F4F4F5F4F0895F6F7909522
:106A70008095709561957F4F8F4F9F4F0895EE0FD2
:106A8000FF1F0590F491E02D09942F923F924F92B1
:106A90005F926F927F928F929F92AF92BF92CF92AE
:106AA000DF92EF92FF920F931F93CF93DF93CDB7B7
:106AB000DEB7CA1BDB0B0FB6F894DEBF0FBECDBF2F
:106AC00009942A88398848885F846E847D848C8400
:106AD0009B84AA84B984C884DF80EE80FD800C8109
:106AE0001B81AA81B981CE0FD11D0FB6F894DEBFEC
:0C6AF0000FBECDBFED010895F894FFCF5C
:106AFC002E003F50313D002650323D002800290029
:106B0C002650333D002650343D002650323D310096
:106B1C0047455420002F20002C2000010000005479
:106B2C005556212223C0A80119C0A80101C0A801F3
:106B3C0001C0A80101FFFFFF00501A4F9033C8326B
:106B4C0040003A00204E0000102700000100020017
:106B5C000000000000000000000000000000000029
:106B6C000000000000000000000000000000000019
:106B7C000000000000000000000000000000000009
:106B8C0000000000000000000000000000000000F9
:106F7C004C6E646B417672613030000A0101000185
:106F8C00500A2C01000001000000002C32D332C248
:086F9C0031F331D3311C320046
:00000001FF
